:020000040800F2
:10000000A0110024A50300089B2300085317000833
:1000100099230008C3160008913200080000000070
:10002000000000000000000000000000112A00088D
:10003000C5160008000000003D290008212B00081B
:10004000BF030008BF030008BF030008BF03000888
:10005000BF030008BF030008BF030008BF03000878
:10006000BF030008BF030008BF030008BF03000868
:10007000BF030008BF030008BF030008BF03000858
:10008000BF030008BF030008BF030008BF03000848
:10009000BF030008BF030008BF030008BF03000838
:1000A000BF030008BF030008BF030008BF03000828
:1000B000692D0008D5300008BF030008BF03000801
:1000C000BF030008BF030008BF030008BF03000808
:1000D000BF030008BF030008BF030008BF030008F8
:1000E000BF030008BF03000800000000BF030008B2
:1000F000BF030008BF030008BF030008BF030008D8
:10010000BF030008BF030008BF030008BF030008C7
:10011000BF030008BF0300084D310008BF030008FB
:10012000BF030008BF030008BF030008BF030008A7
:10013000BF030008BF030008BF030008BF03000897
:1001400000000000000000000000000000000000AF
:10015000BF030008BF030008BF030008BF03000877
:10016000BF030008BF030008BF030008BF03000867
:10017000BF030008BF030008BF030008BF03000857
:10018000BF030008BF030008BF030008BF03000847
:10019000BF030008BF030008BF030008BF03000837
:1001A000BF030008BF030008BF030008BF03000827
:1001B000BF030008BF030008BF030008BF03000817
:1001C000BF030008BF030008BF030008BF03000807
:1001D000BF030008BF030008BF030008BF030008F7
:1001E000BF030008BF030008BF030008BF030008E7
:1001F000BF030008BF030008BF030008BF030008D7
:10020000BF030008BF030008BF030008BF030008C6
:10021000BF030008BF030008BF030008BF030008B6
:10022000BF030008BF030008BF0300080000000070
:10023000BF030008BF03000800000000BF03000860
:10024000BF030008BF030008BF030008BF03000886
:10025000BF030008BF030008BF030008BF03000876
:10026000BF030008BF030008BF030008BF03000866
:10027000BF030008BF030008BF0300080000000020
:10028000BF030008BF030008BF0300080000000010
:1002900000000000BF03000800F002F800F072F850
:1002A0000AA090E8000C82448344AAF10107DA45D1
:1002B00001D100F067F8AFF2090EBAE80F0013F0B1
:1002C000010F18BFFB1A43F001031847D0B200001A
:1002D000F0B200000A444FF0000C10F8013B13F09C
:1002E000070408BF10F8014B1D1108BF10F8015B8F
:1002F000641E05D010F8016B641E01F8016BF9D182
:1003000013F0080F1EBF10F8014BAD1C0C1B09D1D8
:100310006D1E58BF01F801CBFAD505E014F8016B4A
:1003200001F8016B6D1EF9D59142D6D370470000DC
:100330000023002400250026103A28BF78C1FBD8EE
:10034000520728BF30C148BF0B607047662909F0CB
:100350006683642900F0AA80782900F0E38073297D
:1003600000F07584002070471FB509F04EFB00F0C7
:1003700073FC04000020002108F0B6FCE0601FBD03
:1003800010B510BD00F06CFD1146FFF7EDFF05F054
:1003900053F900F08AFD03B4FFF7F2FF03BC00F04D
:1003A000C1FD00000948804709480047FEE7FEE715
:1003B000FEE7FEE7FEE7FEE7FEE7FEE7FEE7FEE715
:1003C00004480549054A064B704700008D2C00087B
:1003D00099020008A00B0024A0110024A00D002405
:1003E000A00D00240FB41CB5074B06AA7B44694638
:1003F0000090059800F001FC0020694600F010FC18
:100400001CBC5DF814FB00003108000070B5044608
:1004100085690068C10601D5302600E02026C007A6
:1004200007D070BDD4E9012130469047206A401CB6
:1004300020626D1EF6D570BD70B5044685690078E2
:10044000C00707D170BDD4E9012120209047206A60
:10045000401C20626D1EF6D570BD70B50C46054679
:10046000012A05D02878800600D5EA69002302E039
:10047000012305E05B1C934202D2E05C0028F9D125
:10048000A869E618C01AA861286A18442862284694
:10049000FFF7BCFF04E0D5E9012114F8010B9047F8
:1004A000B442F8D32846FFF7C7FF70BD2DE9F041ED
:1004B0000646002410687529314616A510D0AFF302
:1004C0000080002802DA404213A507E031688A075D
:1004D00001D512A502E0490704D511A5012401E0C8
:1004E000AFF3008000210A2206F1240709E0B0FBE7
:1004F000F2FCB0FBF2F302FB1C00303078541846DB
:10050000491C0028F3D123462A463046BDE8F04175
:1005100000F005B9000000002D0000002B000000D5
:100520002000000070B504460D4621461068AFF368
:1005300000802188090502D50F4A7A4402E00E4A5C
:100540007A440E32002104F1240305E000F00F0686
:100550000009965D5E54491C0028F7D120780023DD
:10056000000704D5702D02D009B1022311322046B4
:10057000BDE8704000F0D3B8CEA900002DE9F05FCF
:10058000894604464FF0000ADFF824B1FB44C0F866
:1005900020A02046E168884700287DD0252806D085
:1005A000D4E901219047206A401C2062F1E7002530
:1005B0005F462046E16888472028064607DB312E43
:1005C00005D2B81910F8200C08B10543F1E7A807C7
:1005D00001D525F00405C4F81CA00027C4F818A014
:1005E0002A2E09D0304604F0E7FA38B304EB870826
:1005F000303EC8F8186019E059F8041B204604EB97
:1006000087029161E1688847012F064618D1E069A9
:10061000002820DA25F020051DE0D8F8180000EBAE
:10062000800006EB40003038C8F818002046E1682A
:100630008847064604F0C0FA0028EED1012F0AD000
:100640002E2E08D12046E16888477F1C0646022FDF
:1006500045F02005C4DBA069002803DA404245F0DC
:100660000105A061E80701D025F01005A6B1A6F1AB
:100670004100192802D8203645F400654A46314623
:10068000204625604D46FFF761FE60B1012807D086
:10069000ED1D25F0070000E007E000F1080978E70C
:1006A00005F1040975E730467AE7206ABDE8F09F56
:1006B000A4A900004FF0000200B5134694469646E8
:1006C000203922BFA0E80C50A0E80C50B1F1200165
:1006D000BFF4F7AF090728BFA0E80C5048BF0CC013
:1006E0005DF804EB890028BF40F8042B08BF704771
:1006F00048BF20F8022B11F0804F18BF00F8012BE3
:10070000704770477047704710B500F0A9FA00684D
:1007100010BD10B5044600F0A3FA046010BD2DE929
:10072000F0470D4699469246044600F124080168B8
:10073000880604D5E06921F01001216000E0012065
:10074000A84201DD471B00E00027A1697A1902EBEE
:100750000900081AA0612078C00602D42046FFF7DD
:1007600055FE002608E0D4E901211AF8060090475A
:10077000206A401C761C20624E45F4DB2078C006BF
:100780000AD52046FFF742FE06E0D4E901213020D9
:100790009047206A401C2062381EA7F10107F4DC54
:1007A00007E0D4E9012118F805009047206A401CB1
:1007B0002062281EA5F10105F3DC2046FFF73CFE70
:1007C0002078000602D50220BDE8F0870120FBE773
:1007D00070472DE9FF4F0C461E464FF0FF378BB098
:1007E000D2E90001DDF860800A908A46C1F30A551B
:1007F00005B93D46002108464FF00000BAF1000F50
:1008000000F4400005DA00EB80004FF4400101EAFB
:1008100050004FEA9059B9F1010F00DDB9460A982E
:1008200050EA4A000ED044F61050A5F2FF35454379
:100830002F14B8F1000F1ED07542291E1EDDC9F11C
:1008400000021CE0B8F1010F4FF0000001D0302190
:1008500003E0F24305E02154401CB042FBDB30468C
:100860000022002121540B99C1F80880C1E9002021
:100870000FB0BDE8F08FBD1B6D1CDEE74A4600DA05
:10088000694206A800F076FA06AB93E8070003ABCE
:1008900083E8070050460A9900F04BFB8DE80700FB
:1008A000A0F500501F3800900398002D0ADD42F299
:1008B0001F014A460844002303A90390684600F03C
:1008C000B4FD09E0A0F500504A461F38002303A9F3
:1008D0000390684600F0BEFD8DE807000004000CA0
:1008E00003D04FF0FF30410800E01046B8F1000F90
:1008F00003D00022009215461EE0751E05D400F0BC
:10090000B3F9303262556D1EF9D5B3460122084362
:1009100002D000227F1C04E02078302801D1002280
:100920007F1E002A099784D01DE0112D07DA00F000
:100930009BF9303262556D1C50EA0102F5D1084333
:1009400002D00098C8B10EE00021681E05E0235CCB
:10095000625C63542254401E491C8142F7DBAB4663
:10096000A81B401E0990002004F80B000B98099A60
:10097000C0F80880C0E9002B7AE711264FF0000884
:1009800057E72DE9F04F88460446D21D22F00701B3
:1009900091B0D1E90001CDE90A0102F059FD02460A
:1009A0000B98C00F01D02D2007E02068810701D5EA
:1009B0002B2002E0202101EAC000032A099001D087
:1009C000072A05DB03464146204600F093F90BE178
:1009D0002078800601D5E06900E00620B8F1650FB7
:1009E000814606D0B8F1660F18D0B8F1670F70D104
:1009F00031E00020B9F1110F009001DB112301E07B
:100A000009F101030AAA01A90CA8FFF7E2FEDDE93A
:100A10000C70002609F10105834647E001204B4692
:100A200000904FF000470AAA01A90CA8FFF7D1FED9
:100A3000DDE90DB00C995D46002610B909F1010001
:100A40000D18B9EB050003D4C0F1FF3609F101051B
:100A5000A5EB09002BE0B9F1010F01DA4FF0010914
:100A60000020B9F1110F0090484601DD112300E08C
:100A700003460AAA01A90CA8FFF7ABFEDDE90C703A
:100A80004D4600268346207800070AD4AB4500DA9D
:100A90005D4601A8012D04DD411911F8011C302922
:100AA00007D04F4502DA17F1040F04DA012082461D
:100AB0000FE06D1EEEE7002F02DCED1B3E4403E06D
:100AC000781CA84200DD7D1CB81B00F1010A4FF024
:100AD00000472078000703D4AA4501DB4FF0FF3A16
:100AE0000021B7F1004F0DF143088DF8431024D0D9
:100AF00002202B23002F01DA7F422D230A21021E20
:100B0000A0F1010000DC5FB197FBF1FC97FBF1F273
:100B100001FB1C7C17460CF1300C08F801CDEEE708
:100B2000A8F1010003702188090501D5452100E0E5
:100B30006521A0F1010800F8011C09980FA9A1EB9B
:100B40000807FF1D00B10120411901EBEA70A169FE
:100B50003844081A401EA0612078C00602D42046FE
:100B6000FFF754FC099828B1D4E901219047206A85
:100B7000401C20622078C00622D52046FFF746FCA4
:100B80001EE0002E04DBB34502DD01A8805D00E01D
:100B90003020D4E901219047206A401C2062761C55
:100BA000AAF101005FEA000A0AD100F055F8C06816
:100BB0000168405CD4E901219047206A401C206212
:100BC000281EA5F10105DCDC07E0D4E9012118F8B5
:100BD000010B9047206A401C2062381EA7F10107D4
:100BE000F3DC2046FFF728FC032011B041E60000AB
:100BF00001694A1C02610878704700B58FB0CDE9E1
:100C000001310021059105497944CDE903101146D0
:100C10006846FFF7B3FC0FB000BD0000E5FFFFFF23
:100C20000A6802F8010B0A60704710B5436913B1F6
:100C3000AFF3008001E0FFF710FC012010BD127837
:100C400000F124010A7000224A700122EDE71168C8
:100C50004FF0FF32E9E7000000487047600B0024C6
:100C600000487047400B002430B5B0F10A024FEA4B
:100C7000900E71F100034EEA817EB0EB0E0061EB45
:100C800091014FEA101E4EEA017E10EB0E0041EB7F
:100C900011114FEA102E4EEA016E10EB0E0041EBDF
:100CA00011214FEA104E4EEA014E10EB0E0041EBBF
:100CB0001141401841F100014FEAD00040EA417073
:100CC0004FEAD10110EB80054FEA810444EA9074A9
:100CD00044EB01046D1944EB0404521BA3414FF093
:100CE000000348BF0A3200D530BD401C41F100016D
:100CF00030BD00002DE9F0411F460446032601687F
:100D0000072A01F4006004DB08B116A505E016A56A
:100D100003E008B115A500E015A521F01000206042
:100D2000A069C01EA0610FB1401EA0612046FFF760
:100D30006DFB4FB1D4E9012138469047206A401C31
:100D40002062C01C206206E0206AFAE7D4E9012193
:100D500015F8010B9047761EF8D22046FFF76CFB82
:100D6000BDE8F0814E414E006E616E00494E460076
:100D7000696E66002DE9F047814616468AB035480F
:100D800078440DC88DE80D0032487844801C03ACCF
:100D90000DC884E80D0041F69B300844372190FBD4
:100DA000F1F290FBF1F5A5F1800501FB12041B3C6B
:100DB00002D56442012000E00020DFF898A08046C0
:100DC0000027FA44AAF1BE0A0EE0E0070AD0324634
:100DD000684607EB470101230AEB810100F03AFB6B
:100DE0008DE8070064107F1C002CEED1194F7F4462
:100DF000AE3F19E0E80715D007EB04100DF1180A13
:100E000090E80E008AE80E00C068F04201D19819FF
:100E100008903246012306A903A800F01BFB03AB90
:100E200083E807006D10641C002DE3D14FF001032F
:100E300032466946B8F1000F03A802D000F0F5FA77
:100E400001E000F007FBC9E90001C9F808200AB079
:100E5000BDE8F08798A4000000487047400B0024CC
:100E60007546FFF7F9FFAE4605006946534620F088
:100E70000700854618B020B5FFF7A2FABDE820406C
:100E80004FF000064FF000074FF000084FF0000B46
:100E900021F00701AC46ACE8C009ACE8C009ACE8F9
:100EA000C009ACE8C0098D46704710B50446AFF3E1
:100EB00000802046BDE81040FFF76DBA4FF0013CBE
:100EC00050F8042B51F8043B9A4215D1A2EB0C03C5
:100ED000934313EACC130BD150F8042B51F8043B85
:100EE0009A4209D1A2EB0C03934313EACC13E7D047
:100EF0004FF00000704700BFD01A01BAB1FA81F17B
:100F000001F0180122FA01F0CB40C1F12001DBB25F
:100F1000C0B2C01A2CFA01F3D11A914311EAC311DD
:100F2000E6D1704701491820ABBEFEE7260002005B
:100F300070475FEA400C08BF91F0000F4FEA8C2326
:100F40004FEAC12243EA51514FEA1C5018BF00F545
:100F5000F0404FEA300018BF41F000415FEA6C5C9E
:100F600000F02980BCF1FF3F08BF40F0804070478F
:100F7000130C06BF12044FF0100C4FF0000C130EB0
:100F800004BF12020CF1080C130F04BF12010CF184
:100F9000040C930F04BF92000CF1020CD30F04BF9A
:100FA00052000CF1010C11464FF00002A0F11F009D
:100FB000A0EB0C00704711F0004F08BF704731F0F4
:100FC00000413FF4D5AF0B0C06BF09044FF0100CE5
:100FD0004FF0000C0B0E04BF09020CF1080C0B0FB4
:100FE00004BF09010CF1040C8B0F04BF89000CF144
:100FF000020CCB0F04BF49000CF1010CCCF1200313
:10100000A0EB0C0022FA03F302FA0CF241EA03010E
:1010100000F10100704720F07F4C80EA030023F0CC
:101020007F47ACEB070303F57C5300F0004003F16E
:10103000FF032DE980494FEA154B09B44FEA1443E9
:1010400025EA0B4E24EA03480FF2042606EB132789
:1010500049083E785FEA320203FB0667C7F50007DE
:1010600007FB06F64FEA54374FEAD64606F102066A
:1010700007FB066CCCF1005C4FEA1C472CEA074CDE
:1010800007FB06F40CFB06F504EB15464FEA961633
:1010900034BF00204FF000404FEAD13706FB07FC79
:1010A0004FEA1C4C0CFB0BF7D21B03FB0CF761EB5C
:1010B00007010CFB0EF7B0EB074072EB17420CFB7D
:1010C00008F734BFA2EB0742B2EB074261EB1741CE
:1010D0004FEA0C444FEA910706FB07FC4FEA1C4C11
:1010E0000CFB0BF7B0EBC74072EB573203FB0CF76E
:1010F00034BFA2EBC742B2EBC74261EB57310CFBE6
:101100000EF7B0EBC70072EB57720CFB08F734BF59
:10111000A2EBC702B2EBC70261EB5771039F4FEA24
:10112000816141EA921104EBCC044FEAD1374FEAD6
:10113000826206FB07FC42EA90124FEA80604FEAA7
:101140001C4C0CFB0BF7D21B03FB0CF761EB0701EC
:101150000CFB0EF7B0EB074072EB17420CFB08F7E5
:1011600034BFA2EB0742B2EB074261EB17414FEAF3
:101170008C554FEA910704EB9C2406FB07FC4FEAD1
:101180001C4C0CFB0BF7B0EBC74072EB573203FB68
:101190000CF734BFA2EBC742B2EBC74261EB573149
:1011A0000CFB0EF7B0EBC70072EB57720CFB08F7A5
:1011B00034BFA2EBC702B2EBC70261EB577115EB6C
:1011C0004C254FEA816141EA92114FEA82624FEA6F
:1011D000D13742EA901206FB07FC44F100044FEAC3
:1011E00080604FEA1C4C0CFB0BF7D21B03FB0CF787
:1011F00061EB07010CFB0EF7B0EB074072EB1742F7
:101200000CFB08F734BFA2EB0742B2EB074261EBDD
:10121000174115EB1C154FEA813141EA92414FEA23
:10122000823242EA90424FEA80304FEA0C7644F133
:10123000000448EA03434EEA0B484FF0000EB2EBBD
:10124000080C71EB030724BF624639464EEB0E0EC5
:101250004FF0000B0018524149414BEB0B0BB2EB26
:10126000080C71EB03077BF1000B24BF6246394683
:101270004EEB0E0E4FF0000B0018524149414BEB64
:101280000B0BB2EB080C71EB03077BF1000B24BFD7
:10129000624639464EEB0E0E51EA020718BF46F081
:1012A000010616EB0E7655F1000254F1000103D54C
:1012B000BDE88901BDE80088BDE88901BDE80048B6
:1012C000B619524141EB0101A3F10103704780803F
:1012D0007F7E7D7C7B7A7978777676757473727190
:1012E00071706F6E6E6D6C6C6B6A6A696868676648
:1012F00066656464636362616160605F5F5E5E5DDA
:101300005D5C5C5B5B5A5A5959585857575656554D
:1013100055555454535352525251515050504F4FAF
:101320004F4E4E4D4D4D4C4C4C4B4B4B4A4A4A49FF
:101330004949484848474747474646464545454442
:101340004444444343434342424242414141002BCF
:101350009C4630D477002BD01CB54FEA370703B436
:101360004FF010004FF01001BAF1000F06D0BCF1A1
:10137000000FDCBF40F0080040F008014FF0000013
:101380000FBCBDE810400BF1010BBBF1010F08BF12
:101390005FEA170722BF12F1010211F101014FF0BC
:1013A000004143F1000300F0004043EA00007047B1
:1013B000F9D35708D0E746EA064613F1400F4FEA43
:1013C00016461FDD13F1200FDFBF16430A4600212A
:1013D00020335B42BED0C3F1200746EA064602FA3C
:1013E00007F74FEA164646EA0706C3F1200722FA36
:1013F00003F201FA07F721FA03F14FF0000342EA82
:101400000702A7E746EA020646EA06464FEA1646FC
:1014100046EA0106BCBF46EA0646360C4FF000031A
:101420004FF000024FF0000194E72DE9804C9A46FE
:10143000934670B491E8380007C831EA400C48BFC1
:1014400034EA430C03D5FFF7E6FDFFF780FFF0BC5D
:10145000BDE8008C2DE9804C9A46934670B491E823
:10146000380007C810F0804F08BF13F0804F03D139
:1014700000F005F8FFF76BFFF0BCBDE8008C20F032
:101480007F4780EA030023F07F4C07EB0C03A3F5B2
:101490007C5300F00040A3F1FE0392F0000F00F037
:1014A000B38095F0000F00F077802DE901494FEAF5
:1014B00011404FEA144621EA004800FB06FC24EAEA
:1014C000064708FB06F607FB08F800FB07F718EBD2
:1014D00006484CEB164C4FEA124B18EB07484FEA04
:1014E00015464CEB174022EA0B4E0BFB06FC25EA97
:1014F00006470EFB06F607FB0EFE0BFB07F71EEB7F
:10150000064E4CEB164C4FF000061EEB074E4CEB14
:10151000174B18EB0B0840F1000018EB0E0B58EBC3
:10152000000840F100008F1A4FF000013CBFC94392
:10153000661B14BFB5EB040C00213CBFC943F61B6E
:101540004FEA17444EEA8E0E27EA04454FEA1C473D
:1015500004FB07622CEA074C05FB07F70CFB05F6BA
:1015600004FB0CFC16EB074642EB174216EB0C464D
:1015700042EB1C421BEB060658EB0202414146EAD5
:101580009E0601D5BDE80189B619524141EB010122
:10159000A3F10103BDE801894FEA14454FEA114761
:1015A00024EA054621EA074C05FB07F406FB07F78A
:1015B0000CFB06F105FB0CFC11EB074144EB174457
:1015C0004FEA124711EB0C4144EB1C4422EA074C52
:1015D00005FB07F206FB07F70CFB06F605FB0CFC08
:1015E00016EB074642EB174216EB0C4642EB1C4546
:1015F0006A1854F1000148BF7047B619524141EBD7
:101600000101A3F10103704795F0000F37D04FEAB5
:1016100011424FEA144721EA024624EA074C02FB32
:1016200007F106FB07F70CFB06F402FB0CFC14EBBE
:10163000074441EB17414FEA154714EB0C4441EBCB
:101640001C4125EA074C02FB07F506FB07F70CFBDC
:1016500006F602FB0CFC16EB074645EB174516EBAE
:101660000C4645EB1C42121951F1000148BF70476E
:10167000B619524141EB0101A3F1010370474FEA52
:1016800014454FEA114724EA054621EA074C05FBB9
:1016900007F106FB07F70CFB06F24FF0000605FB0F
:1016A0000CFC12EB074241EB174112EB0C4251EBE1
:1016B0001C4148BF7047921841EB0101A3F101039F
:1016C0007047FEE7704700000248C16D816501F078
:1016D000A1B900008000002470B5002400254FF45B
:1016E0007A76284601F08CF92044401CC4B230467A
:1016F00003F028FB6D1CEDB2082DF2D3002001F0A1
:101700007FF90246102001F07BF90244202001F00D
:1017100077F90244302001F073F90244402001F0CF
:101720006FF90244502001F06BF91044C01CC0B2A4
:1017300004B9212418B10021FF2808D000E00121BC
:101740000022114300D04D2444EA002070BD012244
:10175000F7E7FEE770B58020134CA0614FF4967652
:10176000304603F0EFFA4021A161304603F0EAFA77
:10177000304603F0E7FA304603F0E4FA4FF4800510
:10178000A561304603F0DEFA4021A161304603F046
:10179000D9FA6800A061304603F0D4FAA56130465A
:1017A000BDE8704003F0CEBA0004025830B50C4CCE
:1017B0004FF40000A0614FF49675284603F0C2FA7A
:1017C0004021A1610649402018310860284603F0F5
:1017D000B9FA8021A1612846BDE8304003F0B2BAD1
:1017E000000402582DE9F04305460024184E4FF43A
:1017F00000084FF496774FF48009280602D5802020
:10180000B06101E0C6F81880384603F09BFA40202A
:10181000B061384603F096FAC6F818906806050ECF
:10182000641CE4B2082CE8D3384603F08BFA40215C
:10183000B161384603F086FA05481030006840F37D
:10184000C010401CC6F81890C6F81880BDE8F08398
:101850000004025830B50546262D00D9262500245F
:101860000AE004F15A00C1B2042003F0C7FEFF20D1
:1018700007F0FAF8641CE4B2AC42F2D930BD10B5FE
:10188000002404F15A00C1B2042003F0B7FE002086
:1018900007F0EAF8641CE4B2272CF2D310BD000074
:1018A0002DE9F0410025184C184E062122463046FD
:1018B00000F0DEF82146304600F0EBF8B16841F068
:1018C0000101B16000244FF4C877B06840F0040013
:1018D000B060142003F036FA316CA94200DD0D46E9
:1018E000641CBC42F1DBA5F11E00002800DA0020D8
:1018F00007F0F3FC9FED061B53EC112B07F0FCFAED
:10190000BDE8F04107F08CBC0200300400600258D2
:10191000666666666666F63F2DE9F04305460F4645
:101920009046124E3069C007FCD130694FF48039BF
:10193000C00301D5C6F81090F06840F00200F060D6
:1019400000240BE02919285D497800EB0120385369
:10195000642003F0F7F9C6F81090A41C4445F1D3B5
:10196000F06820F00200F060BDE8F0830020005233
:1019700030B500224B68144CA04209D1134CA46826
:10198000C4F30004124DAD68C5F300052C4303E019
:10199000104CA468C4F3000414B10122104630BDF9
:1019A0000D4D53B10C681C43D1E902310B438168E2
:1019B0001C4329400C438460F0E7836809682B408E
:1019C0000B438360EAE7000000230240002002404E
:1019D0000021024000600258E030C0FF30B5002214
:1019E0008368C3F30003002B02D00122104630BDF0
:1019F0008C680B682343C46844F21C05AC43234342
:101A0000C3600369496823F070430B430361EDE74A
:101A100070B500224B688468C4F30004002C02D027
:101A20000122104670BD114D6BB18C680B682343C9
:101A3000D1E90346344323434C692343C4682C4013
:101A40002343C3600AE0CC680B682343D1E9044612
:101A500034432343C4682C402343C3604968036B69
:101A600023F00F030B430363DBE700001CC0F0FF10
:101A700010B501F4407300EB9310036B1F2401F0C9
:101A80001F01C2F384628C408A40A3431343036363
:101A900010BDC2690B030AD091FAA1F1B1FA81F12C
:101AA00001F01F03012199400A43C2617047C1F34D
:101AB0008461F5E710B501F0007300EBD350436982
:101AC0000724C1F304518C408A40A343134343616C
:101AD00010BD000010B550F8C03FC1F31304A3437C
:101AE00002F01804024AE2400A401343036010BDAA
:101AF000FFFF0F0008B504490A6802430A6009683D
:101B00000140009108BD0000E044025808B50449B6
:101B10000A6802430A6009680140009108BD00009C
:101B2000E844025870B5002354680125066801F0A6
:101B300010018D40B54304D0002525B1012318467E
:101B400070BD0125F9E764B1056840F6FC768E406A
:101B5000B54316682643946826438E403543056096
:101B600007E00468FC258D40AC4315688D402C438C
:101B70000460C46B07258D40AC43D2E9035652691B
:101B8000354315438D402C43C463D8E7F0B50A684C
:101B900092FAA2F2B2FA82F453E00123A3401A406F
:101BA000CAB34B68012B01D0022B10D18D681346AC
:101BB00086685B4303EB43076B43BE431E4386606B
:101BC000CD680B6846689E436B431E4346600D69B3
:101BD0001346D0F80CC05B431E4603EB43076B4330
:101BE0002CEA070C4CEA030CC0F80CC04B68022B23
:101BF00020D1FF2A10D84D69D0F820C006FB02F38F
:101C00005343C3EB03126B432CEA020C4CEA030C64
:101C1000C0F820C00EE013E04B69150A05FB05F281
:101C20006A436A43456AC2EB021C5A4325EA0C0523
:101C3000154345624A6803685643BB433343036018
:101C4000641C0A6832FA04F3A7D10020F0BD0069D1
:101C5000814301D000207047012070474FF47A7112
:101C6000B0FBF1F14FF0E020491E4161002181619C
:101C7000052101617047000003490A6822F44032DF
:101C800002430A60704700005844025803490A683A
:101C900022F00F0202430A60704700001844025805
:101CA0000149086070470000140200242DE9F04744
:101CB00002684FF0804A254CDFF89490DFF894C01A
:101CC000A042DFF89480254B09D0504507D0484505
:101CD00005D0604503D0404501D0984203D14D68FE
:101CE00022F070022A431E4D1E4EA0421E4F0FD0FE
:101CF00050450DD048450BD0604509D0404507D030
:101D0000984205D0A84203D0B04201D0B84205D1D4
:101D1000D1F80CC022F4407242EA0C0202608A68D8
:101D2000C2620A888262A04207D0984205D0A842C7
:101D300003D0B04201D0B84201D1096901634169C1
:101D400041F0010141610020BDE8F0870000014041
:101D50000004004000080040000C00400004014066
:101D6000004001400044014000480140034601207A
:101D7000B1F5805F1DD00ADC012912D0102914D0E2
:101D8000B1F5807F1DD11146184600F0BDBBB1F5FD
:101D9000803F12D0B1F5801F13D11146184600F0D4
:101DA0007FBC1146184600F013BB1146184600F0E0
:101DB0005BBB1146184600F0F5BB1146184600F013
:101DC00031BC704708B54FF0E0210A690092421C0F
:101DD00005D0401C03E00A69D20300D5401E00284C
:101DE000F9D108BD30B595B0002412941394149421
:101DF00018210CA8FEF75EFC089409940A940B9431
:101E0000182102A8FEF756FC0020FFF735FF2E48E8
:101E1000016841F020010160006800F0200001909D
:101E20000420FFF767FE032002900390069402A9A6
:101E30002648FFF7ABFE264D296940F20340814357
:101E4000296114201290149412A92846FFF7C6FDA8
:101E50000C940D940E940F9411940CA92846FFF73E
:101E6000D7FD4FF400200890099408A91948FFF7FE
:101E70007FFDA86818490840A860A868174908406D
:101E800040F08050A860164816490068B0FBF1F198
:101E900001EB810040000A21B0FBF1F100E0491E96
:101EA0000029FCD1104C062128462246FFF7E0FD10
:101EB000012221462846FFF7FDFD0C4A214628460F
:101EC000FFF708FE15B030BDD8440258000802588C
:101ED0000020024000230240C0FFFF5FC0FFFF7FE1
:101EE00014020024400D03000004002A0000FF47F4
:101EF00030B58DB000240A940B940C94182104A8DA
:101F0000FEF7D8FB00940194029403940020FFF79D
:101F1000B3FE4FF08070FFF7EDFD0420FFF7EAFD00
:101F20002548016841F040610160244D296940F273
:101F300003408143296118200A900C940AA928467D
:101F4000FFF74CFD0494059406940794099404A9A2
:101F50002846FFF75DFD019469461948FFF708FD23
:101F6000A86818490840A860A8681749084040F0C8
:101F70008050A860154816490068B0FBF1F101EBEC
:101F8000810040000A21B0FBF1F100E0491E002968
:101F9000FCD1104C062128462246FFF769FD00229D
:101FA00021462846FFF786FD40F2FF72214628466B
:101FB000FFF790FD0DB030BD0404005800600258DA
:101FC00000630258C0FFFF5FC0FFFF7F14020024C0
:101FD000400D03000200300410B58CB0182106A893
:101FE000FEF768FB18216846FEF764FB4FF00050CF
:101FF000FFF78CFD0120FFF77DFD302000900320CE
:1020000001900024049415486946FFF7BFFD01F0D4
:1020100045FA0122114600F0C1F90146362001F0CF
:1020200045FA362001F02CFA0694079409940A9494
:102030000B9406AA0B4C0A492046FFF773FD206853
:1020400020F002002060084906AA2046FFF76AFD3A
:10205000206820F4003020600CB010BD0000025851
:102060000100100200740040720040352DE9F04775
:1020700086B018216846FEF71DFB1020FFF73AFDD9
:102080008020FFF737FD0420FFF734FD0120FFF724
:1020900031FD0220FFF72EFD0820FFF72BFD274E14
:1020A0004FF4A810B06148F20919254F4FEA0940D2
:1020B000B8614CF2D81ADFF88C804FEA0A40C8F8B1
:1020C0001800152000900125019500240294039426
:1020D000049469463046FFF759FDCDF8009001950C
:1020E00002940394049469463846FFF74FFD042098
:1020F00000900194049569463846FFF747FD4FF478
:10210000705000900194049569464046FFF73EFDEB
:10211000CDF800A0019502940394049469464046CA
:10212000FFF734FD02200090019404946946304684
:10213000FFF72CFD06B0BDE8F08700000010025844
:1021400000000258000402580B494CF6CC400860CD
:1021500045F2555008600520486040F6FF708860E1
:10216000C868400706D000200128F9D14AF6AA2005
:10217000086070470120F7E70048005810B586B0A6
:10218000142101A8FEF796FA0120FFF7BFFC01F029
:1021900085F90222114600F001F901461C2001F0E8
:1021A00085F91C2001F06CF90020ADF804000290C4
:1021B0000D49039104904FF0804401A92046FFF798
:1021C00075FD206820F080002060A0680749084065
:1021D000A060606820F070006060A06820F080005F
:1021E000A06006B010BD0000804F1200F8BFFEFFD7
:1021F00010B586B0142101A8FEF75CFA0220FFF7A3
:1022000085FC01F04BF90022114600F0C7F80146A9
:102210001D2001F04BF91D2001F032F90020ADF82E
:10222000040002904FF496610391049001A90B4CB5
:102230002046FFF73BFD206820F080002060A0686A
:1022400007490840A060606820F070006060A068E6
:1022500020F08000A06006B010BD00000004004027
:10226000F8BFFEFFF0B593B014210EA8FEF722FAD6
:10227000202106A8FEF71EFA18216846FEF71AFA72
:102280000420FFF743FC0026ADF838600F964FF6A8
:10229000FF70109011960EA9214D2846FFF706FDFC
:1022A000286820F080002860A8681E490840A860BF
:1022B0001D4801781A4818300C18206808211A4F58
:1022C00009373A78914008432060602006900796CD
:1022D000089609960A96012106AA2846FFF746FDA8
:1022E000206804213A78914088432060686820F093
:1022F00070006860A86820F08000A8600820FFF7E0
:10230000F9FBA8140090022001900296039604960F
:10231000059069460548FFF739FC13B0F0BD000091
:1023200000080040F8BFFEFF229A0008000C025887
:1023300010B586B0142101A8FEF7BCF91020FFF7F4
:10234000E5FB01F0ABF80122114600F027F8014649
:10235000362001F0ABF8362001F092F80A20ADF8F3
:102360000400002002904FF6FF700390094C01A971
:102370002046FFF79BFC206820F08000206060680A
:1023800020F070006060A06820F08000A06006B0BF
:1023900010BD000000100040FEE7FEE730B500F081
:1023A0000703C3F10704042C00D90424181D0728CF
:1023B00001D2002300E0DB1E012505FA04F0401ED7
:1023C000084098409D406D1E1540284330BD0000D8
:1023D00030B5026A22F001020262026A436884692F
:1023E00024F003041A4D2C400D682C430D6922F093
:1023F00002022A434D6822F001022A43154DA842E9
:102400000BD0154DA84208D0144DA84205D0144D4C
:10241000A84202D0134DA84212D14D6922F0080201
:1024200042EA85028D6822F0040242EA85028D6943
:1024300023F480732B43CD6923F4007343EA4503EF
:1024400043608461C96841630262002030BD0000BE
:102450008FFFFEFF000001400004014000400140EA
:10246000004401400048014030B5026A22F01002E9
:102470000262046A4268836923F440731C4D2B4056
:102480000D6843EA052524F020030C6943EA041390
:102490004C6823F0100343EA0413164CA0420BD0FF
:1024A000154CA04208D0154CA04205D0144CA042B7
:1024B00002D0144CA04213D14C6923F0800343EAAC
:1024C00084138C6823F0400343EA84138C6922F45C
:1024D000806242EA8402CC6922F4006242EAC402C9
:1024E00042608561C96881630362002030BD0000DD
:1024F000FF8FFFFE0000014000040140004001404A
:10250000004401400048014030B5026A22F4807264
:102510000262036A4268C46924F003041B4D2C4024
:102520000D682C430D6923F4007343EA05234D68BD
:1025300023F4807343EA0523154DA8420BD0154DB3
:10254000A84208D0144DA84205D0144DA84202D08C
:10255000134DA84213D14D6923F4006343EA852348
:102560008D6823F4806343EA85238D6922F48052C9
:1025700042EA0512CD6922F4005242EA4512426055
:10258000C461C968C1630362002030BD8FFFFEFFD4
:1025900000000140000401400040014000440140AF
:1025A0000048014030B5026A22F480520262046A97
:1025B0004268C36923F44073144D2B400D6843EA0D
:1025C00005230D6924F4005444EA05344D6824F4CD
:1025D000805444EA05340E4DA8420BD00D4DA8425C
:1025E00008D00D4DA84205D00C4DA84202D00C4D8C
:1025F000A84204D18D6922F4804242EA85124260E9
:10260000C361C96801640462002030BDFF8FFFFE12
:10261000000001400004014000400140004401402E
:102620000048014030B5026A22F480320262036A37
:10263000426D154C22400C6822430C8A23F400336F
:1026400043EA04438C8823F4803343EA04430F4C69
:10265000A0420BD00E4CA04208D00E4CA04205D098
:102660000D4CA04202D00D4CA04206D144688D69A9
:1026700024F4803444EA052444604265C968826DCC
:1026800081650362002030BD8FFFFEFF0000014026
:102690000004014000400140004401400048014066
:1026A00030B5026A22F480120262026A436D154C50
:1026B00023400C6843EA04230C8A22F4001242EA05
:1026C00004528C8822F4801242EA04520E4CA0423A
:1026D0000BD00E4CA04208D00D4CA04205D00D4CA2
:1026E000A04202D00C4CA04206D144688D6924F46B
:1026F000802444EA852444604365C968C165026258
:10270000002030BDFF8FFFFE0000014000040140AB
:1027100000400140004401400048014070B560495C
:102720000022012603230524072505280ED24E701A
:102730008B70CC700D714A718A71CA710A724A72BB
:102740008A72CA720A734A738A7370BD0ED14A7054
:102750008E70CB700C714D718A71CA710A724A7297
:102760008A72CA720A734A738A7370BD06281ED0B1
:1027700007282BD0082838D0092845D00A2852D05D
:102780000B285FD00C286CD00D287AD00E28ECD105
:102790004A708A70CA700A714A718A71CA710A7263
:1027A0004A728A72CE720B734C738D7370BD4A700D
:1027B0008A70CE700B714C718D71CA710A724A7237
:1027C0008A72CA720A734A738A7370BD4A708A70B9
:1027D000CA700E714B718C71CD710A724A728A7215
:1027E000CA720A734A738A7370BD4A708A70CA705B
:1027F0000A714E718B71CC710D724A728A72CA72F3
:102800000A734A738A7370BD4A708A70CA700A71FB
:102810004A718E71CB710C724D728A72CA720A73D0
:102820004A738A7370BD4A708A70CA700A714A719D
:102830008A71CE710B724C728D72CA720A734A73AE
:102840008A7370BD4A708A70CA700A714A718A713F
:10285000CA710E724B728C72CD720A734A738A738C
:1028600070BD4A708A70CA700A714A718A71CA71E1
:102870000A724E728B72CC720D734A738A7370BD7A
:10288000FFE74A708A70CA700A714A718A71CA7108
:102890000A724A728E72CB720C734D738A73EEE7B2
:1028A0003F02002430B5092800D90920022101EB9C
:1028B0004005C0F10A04F620E9B2604340B205F0D9
:1028C0009DFF04EBC400E9B2BDE8304040B205F022
:1028D00095BF0000164A1748516D0160164B481C01
:1028E000B3FBF0F002F5807340091860052382F80D
:1028F0003B3002F18003586792F82630032B05D253
:1029000040016C2390FBF3F0106604E04001362395
:1029100090FBF3F01066106E20F01F00106650233D
:10292000B0FBF3F050662820B1FBF0F090667047E2
:10293000000000242C040040000E27077047000010
:102940002248016841F400210160016841F0C001A2
:102950000160016841F020010160011F0A6822F452
:102960007C3242F480520A6018490C310A686FF3D5
:10297000080242F011020A600A6822F47E4242F420
:1029800080620A600A6822F4FE0242F480320A6021
:102990000A6822F0FE4242F080720A60091D0A684D
:1029A0004FF6F8739A4342F440420A60016841F0DE
:1029B0001001016005482C38016841F08061016018
:1029C0000168C1F3C0610029FAD070472C44025855
:1029D0000349097A494200EB41400249405C704793
:1029E0000000002400000E080149405C7047000010
:1029F0000000040801480078704700000000060845
:102A00000249084490F800087047000000E0F11FF8
:102A10007047000010B5044CA06D05F091FFA06D4B
:102A2000BDE8104005F058BF8000002410B5084CE8
:102A3000A06D05F085FFA06D05F04EFFA4F18000AC
:102A400090F83A00BDE81040800105F0ADBF0000ED
:102A50008000002470B5403045B20820A0EBD104BE
:102A6000802601F00700C640E9B2E0B202F0C6FDE0
:102A7000054805EB45010144085D3043C0B20855E7
:102A8000BDE8704005F0F0BFD404002470B50E46D8
:102A900008253E2801DD012100E0002110F13E0F54
:102AA00001DA012200E00022114336D1403044B265
:102AB0000820E1B202F0A2FD002005F0D5FF0720BA
:102AC000E1B202F09BFD002005F0CEFF0620E1B24E
:102AD00002F094FD002005F0C7FF072E07D908205B
:102AE000E1B202F08BFDFF2005F0BEFF07250F2E9F
:102AF00007D90720E1B202F081FDFF2005F0B4FF05
:102B00000625E1B2E8B202F079FD044906F00700BB
:102B1000085CBDE8704005F0A7BF70BD1C02002432
:102B20007047000010B55548016821F00F0141F0D1
:102B300002010160016801F00F010229FAD1504839
:102B4000016821F0070141F0020101604C480C309E
:102B5000016821F4404141F400410160494908689D
:102B600040F4803008600868C0F340400028FAD084
:102B700044487430026842F0010202600268C2F305
:102B80004002002AFAD03F4A2832106820F00300A1
:102B900040F002001060101D036843F480330360AE
:102BA000036843F00C030360036823F0020303602F
:102BB000106820F47C7040F0100010603148303014
:102BC00002686FF3080242F03B020260026822F4DE
:102BD0007E4242F400720260026822F4FE0242F475
:102BE00080320260026822F0FE4242F0807202608F
:102BF000086840F0807008600868C0F340600028F2
:102C0000FAD00820FFF742F81E481030016821F082
:102C1000070141F003010160016801F03801182942
:102C2000FAD1184C1834206820F470602060082015
:102C3000FFF72CF8201D016821F0700141F04001E0
:102C40000160016821F4E06141F480610160206865
:102C500020F0700040F0400020600A4820300168F9
:102C600021F0700141F040010160074C2046FEF761
:102C7000F5FF2046BDE81040FFF712B800200052D3
:102C80000C48025800440258001C4E0E10B52C4847
:102C9000016841F4700101602A4A106800F00F00D9
:102CA000072804D2106820F00F00C01D10602649CC
:102CB000086840F001000860234B002010331860C2
:102CC0000B68224C23400B60136803F00F03072BA3
:102CD00004D9136823F00F03DB1D13601A4A18325E
:102CE0001060121D1060121D1060174B184A283317
:102CF0001A601B1D174A1A601B1D174A1A601B1DFC
:102D000018601B1D1A601B1D18601B1D1A601A1D00
:102D100010600A6822F480220A600B496031086062
:102D20000E4800686FF30F00B0F1005F02D20C494B
:102D30000120086043F2D2000A49086010BD00007B
:102D400088ED00E000200052004402587FEDF6EAD2
:102D5000000202020000FF01800201010010005C7D
:102D600008810051004000522DE9F0414FF08041B0
:102D70006FF001000861D14D95F8200000287DD149
:102D80000024DFF83C83002708F1800695F82B101B
:102D900058F82400C1F10201084100EE100A95F82C
:102DA00029102046B8EEC00A02F008FCBDEEC00AA9
:102DB00010EE100A46F8240048F82470641CE4B2AF
:102DC000202CE3D3FF2085F82000E879401CC0B216
:102DD000E87195F8431001290CD140070AD1687AAF
:102DE00000287DD0EA6FC0F10A01B2FBF1F1E9677A
:102DF000401E6872B14C8034676027609FEDB10A55
:102E000084ED1F0A0020B04A02F1800356F820101A
:102E100000EE101AF8EEC00A00EE101AB8EEC01A52
:102E200094ED1F0A00EE810A84ED1F0A00EE101ACD
:102E300002EB800CF8EEC00A94ED000A9CED001A3B
:102E4000B8EEC00A00EE810ABDEEC00A84ED000AA9
:102E500000EE101A03EB8001F8EEC00A94ED010AAF
:102E600091ED001AB8EEC00A00EE810ABDEEC00A6C
:102E700084ED010A401CC0B2202800E08DE0C5D3DB
:102E800094ED1F0ADFED910A20EE200A10EE100AE1
:102E900006F04AFD41EC100B01F032F851EC100B3A
:102EA00005F044FF00EE100A84ED1F0AD5ED190A63
:102EB00095F82B00B8EE601AC0EE010A00EE100A79
:102EC000B8EE400A80EE801ABCEEC10A85ED160A03
:102ED000206820616168616195F83520012A00E071
:102EE00009E003D095F82620032A0AD295F823207A
:102EF0006262226216E076490A6822F001020A60E4
:102F000076E7E269121A00D55242032392FBF3F2EC
:102F1000521C2262A269521A00D5524292FBF3F26D
:102F2000521C6262E269904203DD236A1A44E26144
:102F300002E0236AD21AE261A269914203DD636A68
:102F40001A44A26102E0636AD21AA261EA7F12B156
:102F5000EF77E061A161E269801A2061A269891AB4
:102F6000616195F8261001291CD000EE100AB8EE18
:102F7000C00A02F099F9BDEEC00A84ED0E0A94ED84
:102F8000050AB8EEC00A02F027FABDEEC00A84EDC9
:102F90000F0AA06BA060E06BE060012085F83300B1
:102FA000BDE8F08195F83810012906D0022919D022
:102FB00003292CD004293FD052E000EE100AB8EECD
:102FC000C00A02F027F8BDEEC00A84ED0E0A94EDA7
:102FD000050AB8EEC00A02F0C5F8BDEEC00A84EDDD
:102FE0000F0A3DE000EE100AB8EEC00A02F03CF80D
:102FF000BDEEC00A84ED0E0A94ED050AB8EEC00AD3
:1030000002F0DAF8BDEEC00A84ED0F0A28E000EE07
:10301000100AB8EEC00A02F051F8BDEEC00A84ED05
:103020000E0A94ED050AB8EEC00A02F0EFF8BDEE04
:10303000C00A84ED0F0A13E000EE100AB8EEC00AD1
:1030400001F0BEFFBDEEC00A84ED0E0A94ED050A44
:10305000B8EEC00A02F05CF8BDEEC00A84ED0F0ABB
:1030600095F82A00A0B194ED0E0AB8EEC00A02F05D
:1030700067F9BDEEC00A84ED0E0A94ED0F0AB8EEB2
:10308000C00A02F0F5F9BDEEC00A84ED0F0A80E730
:1030900094ED0E0AB8EEC00A02F006F9BDEEC00AC1
:1030A00084ED0E0A94ED0F0AB8EEC00A02F094F90E
:1030B000BDEEC00A84ED0F0A6BE70000000000249B
:1030C0005003002400000000500200240000003DD6
:1030D0000010004070B517486FF001010160002139
:1030E000154A9078401CC0B29070202800D1917091
:1030F000124B9078124C53F82030236092F8204005
:10310000104B94B1104C1E6C54F8205035446FF4A1
:103110000056354444F82050D06D401CD065146EE4
:10312000A04202D382F82010D165986840F00400D4
:10313000986070BD1004004000000024500400247A
:1031400008740040002002405003002409486FF03A
:1031500001010161084991F84200421C81F84220B6
:10316000C207064802D0002101607047C96F4908B4
:1031700001607047001000400000002414740040FB
:1031800070B51820FFF724FC314D28710520FFF79A
:103190001FFC28701620FFF71BFC68732B3D1420C2
:1031A000FFF716FC05F18004E0651320FFF710FC23
:1031B00018B1E06D00F58070E065FFF72BFC95F825
:1031C0002A000C2248F20101C0B1012819D00126C1
:1031D0000823022818D003281BD00A2604281DD053
:1031E000891C05281FD0062823D0072808D1A166EE
:1031F000EA75A46D0A2C21DB0A3C21E0A166EA7580
:1032000070BDA166EA7570BDA166EB7585F82F608B
:1032100070BD48F20F00A066EE7570BD48F25F0009
:10322000A066EE7570BDA166EB75032085F83800C9
:1032300070BD49F6DF00A066EE7570BD04F5AF7491
:10324000204605F07DFB2046BDE8704005F044BBFC
:103250002B00002410B50C4C012206212046FEF75D
:1032600007FC01212046FEF714FCA06840F0040092
:10327000A0601E2001F066FD206C044991F8311019
:1032800090FBF1F010BD0000006002580000002427
:10329000FEE7000010B5044601F01CFD1C4818A113
:1032A000FDF7A0F81A4A1421032001F011FE4FF493
:1032B000487001F0A9FC012C01D105F0BFFC154CB0
:1032C000207AC0F10700C0B201F04CFE207A202223
:1032D0001149404201EB404104F21110FEF71CFB82
:1032E0000E4801694907FCD4C16841F00101C16081
:1032F00001F0F0FCBDE810406420FEF763BD000063
:10330000202A205752495445202A2020000000003E
:10331000280200240000002400000E0800200052B3
:1033200010B50D4C0B4961600C496160012801D159
:1033300005F0C2FC022001F015FE094920220948CF
:10334000FEF7EAFA20694007FCD4E06840F001008B
:10335000E06010BD2301674500200052AB89EFCD2E
:10336000000004080901002410B5032001F0FAFD53
:10337000064920220648FEF7CFFA064801694907A8
:10338000FCD4C16841F00101C16010BD0000060815
:10339000080000240020005270B506460D46FEF7D6
:1033A000D9F94FF47A74204601F0CCFC5820FEF78E
:1033B00019FA204601F0C6FC3046FEF713FA204603
:1033C00001F0C0FC2846FEF70DFABDE87040FEF79C
:1033D000EDB9000010B50320FFF706FBFF282BD046
:1033E00000220320FFF700FB40B3002002432BD054
:1033F0000520FFF7F9FAFF2822D000220520FFF769
:10340000F3FAF8B1002002431ED0FEF765F90F4928
:1034100066224A7000228A70A1F209139A74040A83
:10342000CC7048710A718A715A675720C8710020A0
:10343000BDE81040FFF774BF0122D2E70120D5E7B5
:103440000122DBE70120DEE710BD000009010024B6
:1034500003B401984100009850EAC12018BF04202D
:103460004A0D18BF40F0010040F2FF72B2EB515F0D
:1034700008BF40F00200012808BF052002B07047D5
:10348000002809DB012100F01F0291404009800063
:1034900000F1E020C0F80011704700000248006809
:1034A000C0F30220704700000CED00E00907090E90
:1034B000002804DB00F1E02080F80014704700F0E1
:1034C0000F0000F1E02080F8141D7047000000009C
:1034D00070B59B482DED020B2DED068B079D25F059
:1034E0000044A04218DC9748844202DC0AD10698C6
:1034F00040B19DED060BBDEC068B02B0BDE87040FF
:1035000001F026BB002DCCBF9FED8F0B9FED900BE4
:10351000BDEC068B02B070BD8F48A04215DD8F4810
:10352000A042D8BF4FF0FF3458DD9DED060B51ECA3
:10353000100BFFF78DFF042808BF01F02DFB9DED58
:10354000060BBDEC068B02B070BD9DED060B51EC79
:10355000100B01F029FDCDE9060181489FED828B1A
:10356000A0423CDD8248A0421FDD00249FED82ABDB
:103570009DED060B53EC1A2B51EC100B05F008FCDB
:103580009DED060B41EC190B53EC1A2B51EC100B73
:1035900005F00AFF53EC182B06F0DCF853EC192B5E
:1035A00005F0AAFCCDE9060149E09DED060B0124DA
:1035B00053EC182B51EC100B05F0EAFB9DED060BBC
:1035C00041EC190B53EC182B51EC100B06F0C2F820
:1035D00053EC192B05F090FCCDE906012FE068486B
:1035E000A0421FDD02249FED689B9DED060B53EC6E
:1035F000192B51EC100B05F0D7FE53EC182B05F0EE
:10360000C7FB9DED060B41EC180B53EC192B51EC4D
:10361000100B06F09FF853EC182B05F06DFCCDE96C
:1036200006010CE09DED060B032453EC102B9FEDDF
:10363000580B51EC100B05F05FFCCDE906019DED38
:10364000060B53EC102B51EC100B05F0ADFE41ECCA
:10365000180B53EC182B05F0A7FE41EC190B4E4844
:103660000621B0EE490AF0EE690A784400F09CFFAA
:1036700053EC182B51EC100B05F096FE41EC180B97
:103680004648B0EE490AF0EE690A0521784400F098
:103690008BFF53EC192B51EC100B05F085FE41EC20
:1036A000100B51EC180B53EC102B002C0EDA05F01C
:1036B0006FFB9DED061B53EC112B05F075FE9DED88
:1036C000061B53EC112B05F06DFF35E005F060FB98
:1036D0009DED061B53EC112B05F066FE41EC100B23
:1036E0002F48784400EBC40090ED001B51EC100B08
:1036F00053EC112B06F02EF89DED061B53EC112B0D
:1037000006F028F841EC100B2648784400EBC40082
:1037100090ED001B51EC100B53EC112B05F042FF08
:1037200041EC100B002DA2BFBDEC068B02B070BDAA
:1037300051EC100B05F0EEFA41EC100B01E7000024
:10374000000010440000F07F182D4454FB21F93F85
:10375000182D4454FB21F9BF0000DC3F0000203E3F
:103760000000F33F00000000000000000000F03FF8
:103770000000E63F000000000000000000000040E4
:103780000080034000000000000000000000F83F3F
:10379000000000000000F0BF7A79000030790000DE
:1037A000BA7800007278000070B56F4E2DED040BF2
:1037B0002DED048B82B0DDF824C0DDE907235C42E7
:1037C0002CF000411C4341EAD474069D22F00040D5
:1037D000B44205D86C422C4340EAD474B4420BD9AD
:1037E0009DED081B9DED060B02B0BDEC048B04B0F3
:1037F000BDE8704001F0B6B9ACF14054A4F17F646B
:103800001C430BD0022404EAAC7444EAD27405438E
:103810009FED578B9FED582B07D015E09DED060BC4
:1038200051EC100B01F0CFF942E0002C11BF012C3C
:103830009DED060B02B0BDEC048B04BF04B070BD5F
:10384000022C38D0032C3BD00B439FED4D1B9FED3A
:103850004E0B0AD0B14218D1B04209D121F08041BB
:1038600020F08040099107900FE0002A15DA10E05F
:10387000474B7B44002C08BF93ED000B0DD0012C6F
:1038800010D0022C17D0032C1AD0B0421DD1002A20
:1038900003DAB0EE410AF0EE610A02B0BDEC048B2F
:1038A00004B070BD93ED000B51EC100B05F032FA33
:1038B00041EC100BF1E7B0EE480AF0EE680AECE7D5
:1038C000B0EE420AF0EE620AE7E7401A00159FEDFB
:1038D000329B3C28C8BF8DED000B17DCBCF1000FFC
:1038E000BCBF10F13C0F8DED009B0FDB9DED080B75
:1038F00053EC102B9DED060B51EC100B05F0FCFA70
:1039000001F052FB01F05FF9CDE90001B4B1012CE7
:1039100010D0022C9FED220B53EC102B9DED000BD1
:1039200051EC100B19D005F015FF53EC182B05F0D6
:1039300011FFBDE7019880F0004001909DED000B64
:1039400053EC192B51EC100B05F02EFC04BF022098
:10395000FCF7DFFE9DED000B9FE705F0FBFE53EC4F
:10396000182B05F01FFEA3E70000F07F0000000009
:10397000182D4454FB210940182D4454FB2109C043
:10398000182D4454FB21F9BF182D4454FB21F93F55
:10399000D2770000000000000000000000000000DE
:1039A000075C143326A6A13C10B52F499FED2C1BB4
:1039B0002DED020B84B0059820F000408842D8BF5E
:1039C0009DED040B2DDD2949884209D1049840B9A9
:1039D0004FF00100FCF79DFE01F0CEF806B010BDDF
:1039E00005DB9DED040B01F0B3F806B010BD684691
:1039F0009DED040B00F004FB10F0030004BF9DEDEF
:103A0000021B9DED000B0CD001280ED09DED021B7A
:103A10009DED000B022817D0012000F041FE06B0FA
:103A200010BD00F009FD06B010BD9DED021B9DED1F
:103A3000000B012000F034FE51EC100B05F06AF988
:103A400006B041EC100B10BD00F0F6FC51EC100B71
:103A500005F060F906B041EC100B10BD000000004D
:103A60000000000000000000FB21E93F0000F07FA3
:103A700070B5D94B00242DED020B2DED108BDDE937
:103A80001010984205DA20F000429A4201D809D17C
:103A900041B19DED100BBDEC108B02B0BDE8704044
:103AA00001F056B8B0F5801F26DA11430BD000287C
:103AB00013DA0120FCF72DFEBDEC108B02B0BDE83F
:103AC000704001F059B80220FCF723FE01F028F8FD
:103AD00051EC100B05F01EF99EE06FF035049FEDE0
:103AE000C00B53EC102B9DED100B51EC100B05F09F
:103AF0005BFCCDE91001084604EB2051C0F3130430
:103B0000B948A1F2FF31204400F4801080F07F62B8
:103B100082F04052224301EB20559FEDB50B1192EC
:103B200053EC102B9DED100B51EC100B05F012FE19
:103B300041EC180BA01CC0F313009FEDAFDB9FED11
:103B4000B0EBB14E7E4403286CD296ED000B51ECE5
:103B5000180B53EC102B05F027FB1DD1002D01BFD6
:103B600096ED000BBDEC108B02B070BD284605F041
:103B7000B4FB41EC180B53EC1D2B05F015FC41EC8C
:103B8000190B53EC1E2B51EC180B05F00DFC53ECEC
:103B9000192B05F0FDF83FE09FED9D0B51EC180B44
:103BA00053EC102B05F000FC9FED9B1B53EC112BED
:103BB00005F0F8FC41EC190B53EC182B51EC180BE9
:103BC00005F0F2FB53EC192B05F0EEFB41EC190B61
:103BD000002D04BF53EC192B51EC180B1AD02846BA
:103BE00005F07BFB41EC1A0B53EC1D2B05F0DCFBC5
:103BF00053EC192B05F0D6FC53EC182B05F0AAFD5D
:103C000041EC180B53EC1E2B51EC1A0B05F0CCFBBE
:103C100053EC182B05F09EFDBDEC108B02B041EC6F
:103C2000100B70BD9FED7E0B51EC180B53EC102B5D
:103C300005F0AEF841EC100B51EC180B53EC102BC7
:103C400005F05AF941EC190B284605F046FB41EC0A
:103C50001B0B53EC192B51EC190B05F0A5FB41EC98
:103C60001A0B714853EC1A2B261851EC1A0B05F05D
:103C70009BFB41EC1F0B6D48C4F1510404F5D724A4
:103C8000B0EE4F0AF0EE6F0A0321784400F08CFC8E
:103C900053EC1F2B51EC100B05F086FB41EC1C0B79
:103CA0006348B0EE4F0AF0EE6F0A0421784400F04A
:103CB0007BFC53EC1A2B51EC100B05F075FB3443D5
:103CC00053EC1C2B05F064F841EC1C0B002C4CDD74
:103CD0009FED510B51EC180B53EC102B05F064FBCE
:103CE00053EC182B05F060FB41EC1A0B55B353EC69
:103CF0001D2B51EC1B0B05F057FB41EC1D0B53EC3E
:103D00001C2B51EC1A0B05F043F853EC192B05F062
:103D10004BFB53EC1D2B05F03BF853EC1A2B05F035
:103D200041FC53EC182B05F015FD41EC180B53EC3E
:103D30001E2B51EC1B0B05F037FB53EC182B05F039
:103D400009FD69E753EC1C2B51EC1A0B05F020F828
:103D500053EC192B05F028FB53EC1A2B05F022FC31
:103D600053EC182B05F01EFC56E735B353EC1D2B16
:103D700051EC1B0B05F018FB41EC1A0B53EC1C2B00
:103D800051EC180B05F0E6FC53EC192B05F00CFB7D
:103D900053EC1A2B05F0DEFC53EC182B05F0DAFC83
:103DA00041EC180B53EC1E2B51EC1B0B05F0FCFAED
:103DB00053EC182B05F0CEFC2EE753EC1C2B51ECEA
:103DC000180B05F0C7FC53EC192B05F0EDFA53EC7A
:103DD000182B05F0E7FB1FE70000F07F0000000054
:103DE0000000000000005043645F09000000000074
:103DF000000000000000F03F763C7935EF39EA3DE5
:103E00000000E0FE422EE63F0075000000000000CA
:103E1000555555555555D53F000000000000E03F71
:103E2000000000000000004086EBF9FFBA720000BD
:103E3000B07200000000000010B52F499FED2C1B50
:103E40002DED020B84B0059820F000408842DCBFC5
:103E500000209DED040B32DD2849884209D10498E9
:103E600040B94FF00100FCF754FC00F085FE06B0AD
:103E700010BD05DB9DED040B00F06AFE06B010BD21
:103E800068469DED040B00F0BBF810F0030011D064
:103E9000012818D09DED021B9DED000B02281AD0C1
:103EA00000F0CAFA51EC100B04F034FF06B041ECFC
:103EB000100B10BD9DED021B9DED000B012000F0CD
:103EC000EFFB06B010BD9DED021B9DED000B00F059
:103ED000B3FA06B010BD012000F0E2FB51EC100B6C
:103EE00004F018FF06B041EC100B10BD00000000FC
:103EF0000000000000000000FB21E93F0000F07F0F
:103F000000B52DED048BB0EE409AF0EE609A83B0D0
:103F100051EC190B05F052FB41EC180B18EE100A8E
:103F200018EE901A8DED008B002818BF0120084371
:103F300020F00040C0F17F6000F1E040C00F14D0DD
:103F400019EE101A19EE900A8DED009B002918BF8A
:103F50000121084320F00040C0F17F6000F1E04003
:103F6000C00F04BF0120FCF7D4FBB0EE480A03B039
:103F7000F0EE680ABDEC048B00BD000000000000FC
:103F800010B51D499FED1A1B2DED020B84B005984D
:103F900020F000408842DCBF01209DED040B21DDB4
:103FA0001649884209D1049840B94FF00100FCF746
:103FB000B0FB00F0E1FD06B010BD05DB9DED040B8C
:103FC00000F0C6FD06B010BD68469DED040B00F084
:103FD00017F800F001000121A1EB40009DED021B4C
:103FE0009DED000B00F0F4FB06B010BD00000000DA
:103FF0000000000000000000FB21E93F0000F07F0E
:104000002DE9F14F04462DED020B2DED088B8AB002
:104010009FEDE70B80ED020B139EE74826F000456D
:1040200085420ADC9DED120B002084ED000B0AB0E6
:10403000BDEC088B03B0BDE8F08FE0489FEDE0AB2E
:104040009FEDE1BBA84247DDE14F9FEDE39B9FED74
:10405000E48B9DED120B53EC1A2B51EC100B002E40
:104060001CDD05F077FB41EC100BBD4208D053EC92
:104070001B2B51EC100B05F06DFBC4E900010BE0AC
:1040800053EC192B51EC100B05F064FB53EC182B7F
:1040900005F060FBC4E900010120C8E704F078FEE8
:1040A00041EC100BBD4208D053EC1B2B51EC100B14
:1040B00004F06EFEC4E900010BE053EC192B51EC47
:1040C000100B04F065FE53EC182B04F061FEC4E9FC
:1040D00000014FF0FF30AAE7C348A84279DB9DED0D
:1040E000120B51EC100B00F05FFF41EC180B9FED31
:1040F000C00B53EC102B05F057F99FEDBF1B53EC91
:10410000112B04F045FE05F08BF8074605F0E5F8A5
:1041100041EC190B53EC1A2B05F046F953EC182B14
:1041200005F040FA41EC180B53EC1B2B51EC190B2A
:1041300005F03AF9DFF8C8A241EC100B4FEA155828
:104140000125FA4453EC102B51EC180B05F002FB3F
:10415000032DC4E900013DD0C1F30A5005EB451120
:10416000A8EB00001139814234DA0AEB051BB0EEEE
:1041700048AA9BED000BF0EE68AA53EC102B51EC13
:10418000190B05F011F941EC1B0B51EC1A0B53EC18
:104190001B2B05F0DFFA41EC180B51EC1A0B53EC1A
:1041A000182B05F0D7FA53EC1B2B05F0D3FA9BED37
:1041B000020B41EC1A0B53EC102B51EC190B05F0D0
:1041C000F3F853EC1A2B05F0C5FA41EC100B6D1CFB
:1041D000B8E70EE0002EA8BF3846BFF628AF94ED32
:1041E000000B51EC100B04F095FDC4E9000178427E
:1041F0001DE7C6F3130040F4801EC6F30A50A0F278
:10420000F530471100F01F05C5F12000DDF848B07A
:1042100008900020069007900520EC467949002D73
:1042200007EB0002794408BF51F8221009D051F879
:10423000223001EB8201AB404A68089922FA01F171
:104240001943A1FB0E26A1FB0B131A449A4234BF5B
:104250000123002303EB06080CEB8003D3E901A63E
:104260000E448E4234BF0121002192448A4411B190
:10427000924502D903E0924501D2012100E00021DC
:10428000C3E901A641444CF82010011EA0F1010031
:10429000C4DC029800F10050850F0298DDE9036745
:1042A0008000DDF8148005F018F841EC1A0B304658
:1042B00005F02AF89FED541B53EC112B05F074F810
:1042C00041EC1B0B384605F01FF89FED511B53ECDA
:1042D000112B05F069F841EC180B404605F014F875
:1042E0009FED4D1B53EC112B05F05EF841EC190BC3
:1042F00051EC180B53EC192B04F04AFD53EC1B2B1B
:1043000004F046FD53EC1A2B04F042FDCDE9080100
:10431000002008909DED080B53EC1A2B51EC100B6C
:1043200005F018FA53EC1B2B05F014FA53EC182B7C
:1043300005F010FA53EC192B05F034F99FED381BFA
:1043400053EC112B05F030F89FED370B41EC180BB7
:1043500053EC102B9DED080B51EC100B05F024F8DD
:1043600053EC182B04F014FD9FED310B41EC180BAE
:1043700053EC102B9DED080B51EC100B05F014F8CD
:1043800053EC182B04F004FD41EC100B139810F0C3
:10439000004F06D06D4251EC100B04F0BBFC41EC19
:1043A000100B284684ED000B41E6000000000000E1
:1043B0000000000000000000FB21E93F7CD9024022
:1043C00000004054FB21F93F3163621A61B4D03DD3
:1043D000FB21F93F000000000000601A61B4D03DED
:1043E0007370032E8A19A33BFB21394100000000A2
:1043F00083C8C96D305FE43F000000000000E03F6B
:104400000A6F0000586E0000000000000000103E1F
:10441000000000000000103C000000000000103A06
:10442000182D4454FB21F93D3326A611460B113CAF
:1044300000000054FB21F93D10B52DED040B2DEDCE
:10444000088B82B0B0EE419AF0EE619A0B9820F0A2
:1044500000449FED4BABB4F1795F11DA9DED0A0B8F
:1044600051EC100B04F0DCFE002801BFB0EE4A0A4C
:10447000F0EE6A0A02B0BDEC088B04BF04B010BDB8
:104480009DED0A0B53EC102B51EC100B04F08CFF3C
:1044900041EC180B3C480621B0EE480AF0EE680AE1
:1044A000784400F081F853EC182B51EC100B04F019
:1044B0007BFF9DED0A0B41EC1B0B53EC192B51ECD0
:1044C000100B04F071FF41EC190B53EC1B2B51EC5A
:1044D000180B04F069FF53EC192B05F03BF99FED25
:1044E0002C0B41EC190B53EC102B51EC180B04F076
:1044F0005BFF41EC100B2848844210DA53EC192B77
:1045000051EC100B05F026F953EC1A2B05F04AF884
:1045100041EC100B02B0BDEC088B04B010BD1F487D
:10452000A042BCBF9FED1E1B8DED001B06DBA4F55A
:1045300000100190002000909DED001B51EC100B2D
:1045400053EC112B05F006F99DED000B41EC180B17
:1045500053EC102B51EC1A0B05F0FCF841EC1A0B44
:1045600053EC192B51EC180B05F0F4F853EC1A2B03
:1045700005F018F841EC100BCCE70000000000003B
:10458000000000000000F03F746B0000000000001D
:10459000000000000000E03F3333D33F0000E93F5C
:1045A000000000000000D23F70B504462DED028BE4
:1045B0004D1E00EBC500B0EE408AF0EE608A90ED33
:1045C000000B35F0060017D053EC182B51EC100BF4
:1045D00004F0EAFE41EC100B6D1E04EBC50090EDFB
:1045E000001B51EC100B53EC112B04F0D1FB41ECF0
:1045F000100B35F00600E7D1022D36D0042D1CD06B
:10460000062D1CBFBDEC028B70BD53EC182B51EC7A
:10461000100B04F0C9FE94ED0A1B53EC112B04F0AF
:10462000B7FB53EC182B04F0BFFE94ED081B53ECC2
:10463000112B04F0ADFB41EC100B53EC182B51EC9B
:10464000100B04F0B1FE94ED061B53EC112B04F09B
:104650009FFB53EC182B04F0A7FE94ED040B53ECD6
:10466000102B04F095FB41EC100B53EC182B51EC84
:10467000100B04F099FE94ED021B53EC112B04F087
:1046800087FB53EC182B04F08FFE94ED001B53ECCA
:10469000112B04F07DFBBDEC028B41EC100B70BDC7
:1046A00031B504462DED040B2DED0A8BB0EE41BA69
:1046B000F0EE61BA0B989DED0A0B20F00040B0F1CE
:1046C000795F0DDA51EC100BFEF7C2FE042808BF2B
:1046D00000F062FA9DED0A0BBDEC0A8B05B030BD0F
:1046E00053EC102B51EC100B04F05EFE41EC180B58
:1046F0009DED0A0B53EC182B51EC100B04F054FEFB
:1047000041EC190B2C48B0EE480AF0EE680A05217E
:104710007844FFF749FF9FED2ACBB0EE40AAF0EEB8
:1047200060AA9CB353EC1C2B51EC190B04F03CFE1B
:1047300041EC1C0B53EC1A2B51EC190B04F034FE1A
:104740009FED210B41EC190B53EC102B51EC1B0B83
:1047500004F02AFE53EC192B04F0FCFF53EC182B49
:1047600004F022FE53EC1B2B04F0F4FF53EC1C2B43
:1047700004F0F0FF9DED0A1B53EC112B04F012FF27
:10478000BDEC0A8B05B041EC100B30BDFFE753ECDC
:104790001A2B51EC180B04F007FE53EC1C2B04F001
:1047A000F7FA53EC192B04F0FFFD9DED0A1B53ECB7
:1047B000112B04F0EDFAE3E7046A000000000000AA
:1047C000495555555555C5BF000000000000E03F54
:1047D000F1B506462DED040BBD482DED0C8B8AB0CE
:1047E000B0EE418AF0EE618A179D25F000449FEDFE
:1047F000BABB9FEDBBCB844208DA9DED160B51ECA2
:10480000100B04F00DFD002800F0E980B64FA74220
:1048100031DC002D0DDA9DED160B51EC100B04F080
:1048200079FACDE9160151EC180B04F073FA41EC5A
:10483000180B9FEDAF0B53EC102B9DED160B51ECAD
:10484000100B04F0AFFE53EC182B9FEDAB0BCDE932
:10485000040151EC100B04F07DFF41EC100B53EC04
:10486000102B9DED040B51EC100B04F091FA9FED11
:10487000A48BCDE916019DED160B53EC102B51ECDA
:10488000100B04F091FDCDE904019DED040B53ECF8
:10489000102B51EC100B04F087FD41EC190B9A48DA
:1048A0000621B0EE490AF0EE690A7844FFF77CFE73
:1048B0009648B0EE40DAF0EE60DAB0EE490AF0EE7B
:1048C000690A06217844FFF76FFE9DED041B51EC49
:1048D000100B53EC112B04F067FD9DED040B41EC24
:1048E0001A0B53EC102B9DED160B51EC100B04F032
:1048F0005BFD41EC190B53EC1A2B51EC1D0B04F032
:1049000047FA53EC192B04F04FFD53EC182B04F02D
:104910003FFA9DED041B53EC112B04F045FD53ECC5
:10492000182B04F035FA41EC180B9FED790B51EC84
:10493000190B53EC102B04F037FD53EC182B04F03B
:1049400027FA41EC190B9DED160B53EC192B51EC8A
:10495000100B04F01DFA41EC180BA74269DC30463D
:1049600004F0BBFC41EC1A0B51EC180B53EC1A2B66
:1049700004F00EFA41EC1B0B53EC182B51EC180B06
:1049800004F012FD53EC1B2B04F0B6FA53EC192B78
:1049900004F0E0FE9DED161B53EC112B04F002FE1B
:1049A0009FED5D1B53EC112B04F0FEFC53EC1A2B16
:1049B00004F0F8FD41EC180B022000EAA570C0F1EC
:1049C000010004F08AFC53EC182B04F0EDFC00BF4E
:1049D00041EC100B0AB0BDEC0C8B05B0F0BD711CA6
:1049E0001698214308430CD09DED160B012E1CBFD9
:1049F00053EC102B51EC1C0B10D000BF04F07CFAD0
:104A0000E6E79DED160B51EC100B00F0CDFA41ECF2
:104A1000100B51EC1B0B53EC102BEFE751EC100B70
:104A2000FEF716FD042808BF00F0B6F89DED160B42
:104A3000D0E7012E04BFB0EE480AF0EE680AC9D0F4
:104A40008DED048B002404949DED040B53EC102B8E
:104A50009DED160B51EC100B04F0A4FD53EC192B3B
:104A600004F0A0FD41EC190B53EC182B51EC1C0B7E
:104A700004F042FA41EC180B8DED008B00949DED93
:104A8000040B53EC102B9DED000B51EC100B04F0BC
:104A90008BFC53EC1B2B04F07BF99DED000B41ECE0
:104AA0001A0B53EC192B51EC100B04F07DFC53EC5A
:104AB0001A2B04F06DF953EC182B04F075FC9DEDE6
:104AC000001B53EC112B04F063F981E70000000098
:104AD0000000303E00000000000000000000F03F39
:104AE000000000000000F0BF2894E53F0000000037
:104AF000182D4454FB21E93F075C143326A6813C62
:104B0000000000000000000092680000A86800009B
:104B1000635555555555D53F000000000000004035
:104B20009FED070B10B553EC102B9FED070B51ECCD
:104B3000100B04F0E1F941EC100B10BD0000000077
:104B40000000000000000000000000000000F03F36
:104B500010B553EC102B51EC100B04F019F941EC8B
:104B6000100B10BD10B553EC112B51EC100B04F0D1
:104B70000FF941EC100B10BD9FED050B10B553EC78
:104B8000102B51EC100B04F0B7F941EC100B10BDD9
:104B900000000000000000009FED050B10B553EC75
:104BA000102B51EC100B04F0FFFB41EC100B10BD6F
:104BB000000000000000001030380A2801D2012057
:104BC00070470020704710B541EC100BFEF780FCD9
:104BD00051EC100B10BD0000084A92F837309B00D2
:104BE0004B43D3670649B1FBF0F10648C162092186
:104BF0005172016841F0010101607047000000241A
:104C0000808D5B000010004010B50D49002281F836
:104C10004320162391F8362012FB03F2CA67094994
:104C2000094CB1FBF0F0E062206840F00100206028
:104C30006E20FDF7C7F8206820F00100206010BD4D
:104C400000000024808D5B00001000402DE9F04141
:104C5000114D95F8231003291BD095F837108906BC
:104C60000E0E0E490E4FB1FBF0F0F862386840F0BE
:104C700001003860082406FB04F0E8671E20FDF7F9
:104C8000A1F8641EE4B2002CF5D1386820F00100D0
:104C90003860BDE8F081000000000024808D5B00DA
:104CA0000010004010B50021094C0022002001EB4B
:104CB000410323441A54401CC0B20428FAD3491CAF
:104CC000C9B28129F2D33F2084F8C00010BD000092
:104CD000D4040024F0B54FF400470B4E3804B06103
:104CE00000256D1C0121E8B200F088FC00240020A2
:104CF00003F0BAFE641CE4B2842CF8D3EDB2092DA3
:104D0000EFD3B761F0BD000000040258F0B54FF4D6
:104D100000470B4E3804B06106250121284600F0FB
:104D20006DFC0024002003F09FFE641CE4B2842C80
:104D3000F8D36D1CEDB2092DEFD3B761F0BD0000C3
:104D40000004025810B50146491EFDD10246521E0C
:104D5000FDD103465B1EFDD10446641EFDD1401EFD
:104D6000FDD110BD002204E00021491C6E29FCD3B6
:104D7000521C8242F8D370472DE9F04F8146884695
:104D80009246002617494FF00040886123E02F38F3
:104D9000C0B200251449C0EB001001EBC00741462A
:104DA00009EB0500C0B200F029FC002405EB450B1F
:104DB00004EBCB00385C03F057FE641CE4B2182C03
:104DC000F6D36D1CEDB2052DE9D3761CF6B208F1D1
:104DD000180808F0FF081AF806000028D7D1BDE827
:104DE000F08F000000040258349A00082DE9F04FBB
:104DF000814688469246002618494FF00040886157
:104E000025E02F38C0B200251549C0EB001001EB9A
:104E1000C007414609EB0500C0B200F0EFFB0024DB
:104E200005EB450B04EBCB00385CC043C0B203F08C
:104E30001BFE641CE4B2182CF4D36D1CEDB2052DDE
:104E4000E7D3761CF6B208F1180808F0FF081AF844
:104E500006000028D5D1BDE8F08F000000040258FC
:104E6000349A00082DE9F04782460F469146002506
:104E700015494FF00040886199F80000802802D25F
:104E80004FF0200819E04FF0610816E0A0EB080091
:104E9000C6B23946504600F0B1FB00240B4906EB80
:104EA00086004618305D03F0DFFD641CE4B2052C7B
:104EB000F8D36D1CEDB2BF1DFFB219F80500002834
:104EC000E4D1BDE8F087000000040258C4AA00083D
:104ED0002DE9F04F8146884693460026B9F1000F30
:104EE00039D01E494FF0004088619BF800008028AF
:104EF00002D24FF0200A2AE04FF0610A27E0A0F129
:104F00002001DE2921D8A0EB0A00C0B200251449F7
:104F100001EB0017414609EB0500C0B200F06EFB43
:104F2000002404EBC500385C03F09EFD641CE4B271
:104F3000082CF6D36D1CEDB2022DEBD3761CF6B225
:104F400008F1080808F0FF0801E0761CF6B21BF82B
:104F500006000028D3D1BDE8F08F000000040258FD
:104F6000C4A00008092818D80C49CA68D20703D081
:104F70000B4A4A600B4A4A60CA6822F4E06242EA7D
:104F80000020C860C86840F00400C860C86840F0ED
:104F90008000C8600220FCF715BF70470020005257
:104FA00023016745AB89EFCD82B0CDE9000121F047
:104FB000004001909DED000B02B051EC100B7047CA
:104FC000B0EE401A9FED100A1E20104A411E02EB5F
:104FD000800002EB8103D3ED000AC0ED000AC8B2E5
:104FE0000028F3D182ED001A094901EB8003D3EDCB
:104FF000000A02EB800393ED001A00EE810A401CC8
:10500000C0B21F28F1D370470000000054060024EE
:10501000E4AD0008B0EE401A9FED100A0A20104AD5
:10502000411E02EB800002EB8103D3ED000AC0EDCC
:10503000000AC8B20028F3D182ED001A094901EB39
:105040008003D3ED000A02EB800393ED001A00EE1B
:10505000810A401CC0B20B28F1D370470000000049
:105060004C07002460AE0008B0EE401A9FED100A15
:105070000820104A411E02EB800002EB8103D3EDB1
:10508000000AC0ED000AC8B20028F3D182ED001A70
:10509000094901EB8003D3ED000A02EB800393ED95
:1050A000001A00EE810A401CC0B20928F1D37047F3
:1050B00000000000D00700248CAE0008B0EE401ABB
:1050C0009FED100A0620104A411E02EB800002EB01
:1050D0008103D3ED000AC0ED000AC8B20028F3D165
:1050E00082ED001A094901EB8003D3ED000A02EBBF
:1050F000800393ED001A00EE810A401CC0B207281D
:10510000F1D37047000000003C080024B0AE000856
:10511000B0EE401A9FED100A1E20104A411E02EB0D
:10512000800002EB8103D3ED000AC0ED000AC8B293
:105130000028F3D182ED001A094901EB8003D3ED79
:10514000000A02EB800393ED001A00EE810A401C76
:10515000C0B21F28F1D3704700000000D006002421
:10516000E4AD0008B0EE401A9FED100A0A20104A84
:10517000411E02EB800002EB8103D3ED000AC0ED7B
:10518000000AC8B20028F3D182ED001A094901EBE8
:105190008003D3ED000A02EB800393ED001A00EECA
:1051A000810A401CC0B20B28F1D3704700000000F8
:1051B0007807002460AE0008B0EE401A9FED100A98
:1051C0000820104A411E02EB800002EB8103D3ED60
:1051D000000AC0ED000AC8B20028F3D182ED001A1F
:1051E000094901EB8003D3ED000A02EB800393ED44
:1051F000001A00EE810A401CC0B20928F1D37047A2
:1052000000000000F40700248CAE0008B0EE401A45
:105210009FED100A0620104A411E02EB800002EBAF
:105220008103D3ED000AC0ED000AC8B20028F3D113
:1052300082ED001A094901EB8003D3ED000A02EB6D
:10524000800393ED001A00EE810A401CC0B20728CB
:10525000F1D370470000000058080024B0AE0008E9
:10526000C0F30721C0B211FB001200F1110111447B
:1052700001FB00120D301044C0B24FF6FF7202EA7B
:1052800001210844704730B502460C4601251146FD
:1052900005EBD40000F0B2F904F007008540E8B255
:1052A000BDE8304003F0E0BB30B50320214BA3F153
:1052B0001002411E03EB8104D4ED000A03EB8004CD
:1052C000C4ED000A02EB810402EB8000D4ED000A79
:1052D000C0ED000AC8B20028EBD183ED000ADFED73
:1052E000160A20EE200A82ED000A0120134901F17E
:1052F000100401EB800595ED000A03EB8005D5ED68
:10530000000A04EB800520EE200AD5ED000A02EB2E
:10531000800595ED001A00EEC10AD2ED000A30EECC
:10532000200A82ED000A401CC0B20328E1D992EDA8
:10533000000A30BDA80A00245BC0FF3CCCAE0008C8
:1053400030B50320214BA3F11002411E03EB810471
:10535000D4ED000A03EB8004C4ED000A02EB8104E3
:1053600002EB8000D4ED000AC0ED000AC8B20028AC
:10537000EBD183ED000ADFED160A20EE200A82ED64
:10538000000A0120134901F1100401EB800595ED9D
:10539000000A03EB8005D5ED000A04EB800520EE42
:1053A000200AD5ED000A02EB800595ED001A00EE0B
:1053B000C10AD2ED000A30EE200A82ED000A401C3C
:1053C000C0B20328E1D992ED000A30BDE80A0024FA
:1053D00010D2AC3EECAE000830B50320214BA3F157
:1053E0001002411E03EB8104D4ED000A03EB80049C
:1053F000C4ED000A02EB810402EB8000D4ED000A48
:10540000C0ED000AC8B20028EBD183ED000ADFED41
:10541000160A20EE200A82ED000A0120134901F14C
:10542000100401EB800595ED000A03EB8005D5ED36
:10543000000A04EB800520EE200AD5ED000A02EBFD
:10544000800595ED001A00EEC10AD2ED000A30EE9B
:10545000200A82ED000A401CC0B20328E1D992ED77
:10546000000A30BDC80A00245BC0FF3CCCAE000877
:1054700030B50320214BA3F11002411E03EB810440
:10548000D4ED000A03EB8004C4ED000A02EB8104B2
:1054900002EB8000D4ED000AC0ED000AC8B200287B
:1054A000EBD183ED000ADFED160A20EE200A82ED33
:1054B000000A0120134901F1100401EB800595ED6C
:1054C000000A03EB8005D5ED000A04EB800520EE11
:1054D000200AD5ED000A02EB800595ED001A00EEDA
:1054E000C10AD2ED000A30EE200A82ED000A401C0B
:1054F000C0B20328E1D992ED000A30BD080B0024A8
:1055000010D2AC3EECAE000870B54FF40046204C13
:105510003004A061C50D1F4BC0099861C820FFF77A
:1055200021FC9D612820FFF71DFCE22003F07CFA9E
:105530001420FFF717FC2C2003F076FA1420FFF755
:1055400011FC2E2003F070FA1420FFF70BFC2F2023
:1055500003F06AFA1420FFF705FC252003F064FA33
:10556000812003F061FA282003F05EFAA22003F004
:105570005BFAC82003F058FAA02003F055FA402047
:1055800003F052FAAF2003F04FFAA66170BD00009D
:10559000000402580000025810B502F0AFFFFDF7FA
:1055A00099F9FDF7EDFD044890F82B00FCF78CF815
:1055B000BDE81040FDF73ABA00000024C1F10B012C
:1055C00000EE901AF3EE0E1AF8EEE00A80EEA11A41
:1055D0000949F7EE000A01EB8000D0ED001A70EEE9
:1055E000C10A60EEA10A41EE000AC0ED000ABDEE5C
:1055F000E00AB8EEC00A70479008002410B50B4BC3
:105600004FF000429A61491ECCB2401EB030C0B289
:1056100003F00AFA102000EB141003F005FA04F06E
:105620000F00BDE8104003F0FFB90000000402586D
:105630004000FCF7C7BB00002DED068B84B0FE4890
:10564000016841F002010160006800F00200019071
:10565000FA4908684FF6FF021040F94A40F44070DA
:1056600010430860FDF71AFF00220F21FCF796FE99
:1056700001464FF0FF30FDF719FFFDF753FAFDF734
:105680005FF9FCF7F3FCFCF7ADFBFCF731FCFCF732
:1056900075FDFCF7ADFDFCF79FFCFCF7E3FDFCF7A7
:1056A00047FEFCF751FD72B6C820FFF7C1FF01208D
:1056B000E4498861FFF728FFFFF70CFB4FF08040BB
:1056C000016821F002010160C16841F00101C1607F
:1056D000016841F001010160DB48016821F002012D
:1056E0000160C16841F00101C160016841F0010140
:1056F0000160D64C206820F002002060206A40F053
:1057000001002062206840F001002060D048606302
:10571000D048016821F002010160C16841F0010137
:10572000C160016841F001010160CB4DA86840F003
:105730008040A8601420FCF745FBA86840F00040BA
:10574000A860A8680028FCDB1420FCF73BFBC34ED4
:10575000B06840F00040B060B0680028FCDB142066
:10576000FCF730FBBE492846FCF793F9BD492846B3
:10577000FCF78FF9AA68BC490A40521CAA60B068BD
:105780000840401CB060B948016841F00101016067
:10579000016841F480310160C820FCF713FB40F63A
:1057A000AC5060630020FDF713F9B14DFF28DFF81E
:1057B000C4924FF400664FF0000B0ED071102846D3
:1057C000FCF745FAE0B931462846FCF740FAB8B98B
:1057D00071002846FCF73BFA90B989F808B0002020
:1057E000FDF758FD99F80800401CC0B289F8080080
:1057F0000428F4D389F808B09E480830FDF7B4FDBA
:10580000FDF7F8F889F80800032802D9032089F881
:105810000800FFF7C1FE99F830004FF4C86110FB93
:1058200001F08A494863012089F8260089F825B0EB
:105830006420FCF7C7FA99F81A00012869D04FF4E0
:105840008040A86104207F49886102F057FE62B65B
:105850006420FCF7B7FA8A4887A1FAF7C3FD05244C
:105860000120214687A2FFF733FB40F6B830FFF74F
:10587000CBF91521022084A2FFF72AFB4FF4FA602E
:10588000FFF7C2F92521012080A2FFF721FB4FF489
:105890007A70FFF7B9F9352102207DA2FFF718FBD6
:1058A0006420FCF78FFA422101207AA2FFF710FB57
:1058B00040F2DC5A5046FFF7A7F93220FCF782FA93
:1058C0005046FFF7A1F96E4875A278A1FAF78AFD54
:1058D0006B4A41210320FFF7C5FA4FF4C870FCF76B
:1058E00071FA0C2089F81D00D9F87000FFF7B8FC98
:1058F000D9F8741088421AD1FBF7EEFED9F870106F
:10590000884214D1042089F83D00022089F83C0027
:105910002DE04FF08040A8614A4900138861C820FB
:10592000FFF786FE99F8190002F03CFF8DE704208E
:1059300089F83D00012089F83C00FFF7E5FDFFF7FD
:10594000C9F94F485AA1FAF74DFD4D4A18210120D7
:10595000FFF7BEFA4A4859A1FAF744FD484A0A211E
:105960000320FFF7B5FA4FF47A70FFF761FE99F85C
:10597000130055281ED099F83C0002281AD1FBF7D5
:105980008FFF99F85810484300F00700062811D1FE
:10599000FFF7A0F93A484DA1FAF724FD384A0A2149
:1059A0000320FFF795FA41F28830FFF741FE4FF4EC
:1059B0000010A86199F83C00022806D099F82C0044
:1059C000142802D9142089F82C0029484FF40061CA
:1059D000FCF73DF938B9264E4FF48065294630462C
:1059E000FCF735F930B122484FF40051FCF72FF99C
:1059F00000B332E1FF2089F805000F2089F8250067
:105A0000012089F80600FFF765F91D4833A1FAF770
:105A1000E9FC01211A4A0846FFF75AFA2820C9F87A
:105A2000780040F6B830FFF7EFF829463046FCF72B
:105A30000EF95DE05FE00000F44402580CED00E078
:105A40000000FA0500100258000400400008004061
:105A5000905F0100001000400020024000600258EA
:105A60000004002A0008302EC0FFFF7F00740040B1
:105A700000040258000000244B504F542D00000039
:105A8000280200244B000000500000004F000000DE
:105A90005400000053544D2D3C48373E2000000078
:105AA0007631342F30342F32360000002573200039
:105AB0002A2A2A44454D4F2A2A2A00007261646925
:105AC0006F646F6D40692E7561000000204B455971
:105AD000204552524F52212000000000466163745D
:105AE0006F72792073657474696E677300000000CB
:105AF00000289AD04EE1FFF7EDF8FF48FAA1FAF737
:105B000071FCFD4A02210120FFF7ACF9012089F860
:105B100021000A2089F83A00FCF788FF40F6E445A6
:105B20006420FFF785FD4FF41C74F44804601420D2
:105B3000FFF77EFDD9F85800A84201D205462E464F
:105B40000A3C952CF1DC99F82B006FF0360110FB24
:105B500001F006EB400001909FEDE98B9FEDEA9B81
:105B600000266420FFF764FD4FF41C75E3480560D0
:105B70001420FFF75DFDD9F85800B04204D906465D
:105B8000A8462321B0FBF1FA0199411A99F82B009C
:105B9000C0EB00104000B1FBF0F43C2C00D93C24D9
:105BA000C5F51C7003F099FBB0EE481AF0EE681AC8
:105BB00053EC112B03F0A0F9B0EE491AF0EE691A7C
:105BC00053EC112B03F0C6FD03F02AFB40B2E1B207
:105BD000FCF740FFD9F858302320CD496A1CB3FBAD
:105BE000F0F091FBF2F2CBA10090C348FAF7FAFB78
:105BF000C14A02210120FFF735F9CB494AF6AA2014
:105C000008606D1E952DB1DAC14908F10100CDF88B
:105C100000A091FBF0F399F82B20C4A1B648FAF745
:105C2000E1FBB54A02210120FFF71CF94FF40055B2
:105C3000C34CEE1005E031462046FCF708F800287A
:105C40008ED029462046FCF702F80028F3D1FFF752
:105C5000A3FCB5494AF6AA20086000241C2120466E
:105C6000FFF711FB641CE4B2802CF7D399F82A10DB
:105C700099F8010000EB4101B24850F82120B2A18F
:105C80009D48FAF7AFFB9C4A19210520FFF720F940
:105C900099F81A0001280AD199F81920ABA1964861
:105CA000FAF7A0FB944A0F210720FFF711F94FF4F0
:105CB000FA752846FCF786F80C2089F81D00A048E4
:105CC0004FF48051FBF7C3FFF0BB2846FEF79CFF63
:105CD000FFF700F8FBF7E4FD039040F6E445DFF83A
:105CE0007CA24AF6AA26DFF84082C820FFF7A0FC73
:105CF000C8F80060D9F85800A84201D9C9F858502E
:105D000097A1039B7C48DAF87420FAF76BFB7A4A78
:105D100003210120FFF7DCF8774895A1D9F8582036
:105D2000FAF760FB744A03210420FFF725F8724854
:105D300090A1FAF757FB704A64210720FFF7C8F8D3
:105D40007F484FF4005100E007E0FBF780FF002898
:105D5000CBD14FF4C870FEF757FF6420FFF768FC03
:105D6000FBF79EFD052813DAFEF7B4FF624882A117
:105D7000FAF738FB604A14210320FFF7A9F8322014
:105D8000FEF742FF3C20FEF73FFF6420FFF750FC88
:105D9000FDF760FA714E0125803EF5774FF47A7079
:105DA000FCF710F8FEF796FF96F83C00401DF076E1
:105DB0009FED758B694E543E3078C0F11E007070B7
:105DC000DFF8988198ED020A88ED0A0AD8ED030AF7
:105DD000C8ED0C0AB0792C3E00287CD0306D03F061
:105DE000A3FD41EC100BFEF727F8D8F83000B0EE19
:105DF000409AF0EE609A03F070FA53EC192B03F01E
:105E0000D3FA41EC1A0B306D03F08EFD41EC100B10
:105E1000FDF7CAFDD8F82800B0EE409AF0EE609A7F
:105E200003F05BFA53EC192B03F0BEFA53EC1A2B78
:105E300002F0AEFF03F0F4F9C8F84000306D03F053
:105E400073FD41EC100BFDF7F7FFD8F82800B0EE1A
:105E5000409AF0EE609A03F040FA53EC192B03F0ED
:105E6000A3FA41EC1A0B306D03F05EFD41EC100B10
:105E7000FDF79AFDD8F83000B0EE409AF0EE609A47
:105E800003F02BFA53EC192B03F08EFA53EC1A2B78
:105E900003F060FC03F0C4F9C8F84400C8F84800F7
:105EA00096F82A0004281ED06420C8F86400D8F8A8
:105EB0004800C01C03F011FA41EC100BFDF7D8FDAF
:105EC0009FED331B51EC100B53EC112B03F014F826
:105ED00003F0A6F900E0A2E0C8F86000002801DAAB
:105EE000C8F860B058E0ABE020202020202020201F
:105EF0002057616974212000280200242C040040EE
:105F00006666666666660E4000000000000050404F
:105F1000703839002564487A2025646D42204B553D
:105F20003D2564202020200000480058472564209B
:105F30004D41583D2564487A204B553D256420004D
:105F400000040258D401002425730000464D202D82
:105F5000202564206D487A20000000008000002485
:105F60002564487A202A2025646D41200000000025
:105F700025642F006D562000205475726E20636FCB
:105F8000696C2120000000006666666666A64C40CB
:105F9000000000606666F63FD8F84800C11700EBC5
:105FA00091704FEAA0094AF6E03081450DDD0621E7
:105FB000C320FEF711FE49F64040FEF7C3FE06215E
:105FC000C320FEF709FE86F833B096F94610D8F8DC
:105FD00060000844C1B286F8221096F83320012AE6
:105FE00034D04FF49670FEF7ADFE96F82700DC280B
:105FF0007ED0002196F82820DC2A7AD00022114396
:106000000AD0C8F86CB086F80DB086F80CB0717C78
:106010007174F57786F845B0C2286BD0FFE1B8EE11
:10602000E01AF8EEC01A96ED142A01EEC21ABDEE7F
:10603000C11A88ED121A88ED100AC8ED110A2FE76F
:10604000D8F828004010C8F8640030E786F833B06C
:1060500096F82620012A60D0022A7CD0491C4FF4F1
:10606000FA70C9B2FEF7B8FD96F82D10D8F84800BE
:10607000884271DDD8F86420B2EB410FF9DDC82801
:1060800001DD86F8345086F827B096F82800401CC9
:10609000C0B286F82800322800D9F577D8F82C103D
:1060A000D8F84000401AC8F84000D8F83420D8F892
:1060B0004410891AC8F8441000EE101AF8EEC00A0D
:1060C00000EE100AB8EEC00A02F0F0FC40B23073E5
:1060D000D8F878100144C8F87810D8F84810B942B8
:1060E00003DDB073C8F86C900F46B07B307402E0EB
:1060F0008FE190E191E1307396F8380096F828200E
:10610000401D82427FF671AF01EBD170401002F06A
:10611000C1FB6420FEF716FE67E796F82D00D8F85D
:106120004810421C914259DDD8F86410814255DD77
:1061300086F844B086F827B096F82800401CC0B214
:1061400086F82800142800D9F577D8F82C10D8F84C
:106150004000401A01E0E1E02AE1C8F84000D8F828
:106160003420D8F84410891AC8F8441000EE101AE8
:10617000F8EEC00A00EE100AB8EEC00A02F096FC73
:1061800040B230737074D8F84810B94203DDB07370
:10619000C8F86C900F4696F91020904200DAF07320
:1061A000F07B307496F90E00307396F8362086F83E
:1061B000372096F82320022A0DD164290BDD96F9A9
:1061C0004510072907DD0A2805DD4FF4FA60FEF7C0
:1061D0003DFD86F845B002F02BFA06E70027642063
:1061E00006F80F0F307E401C307686F819B0D8F8CC
:1061F0004000C8F82C00D8F84400C8F83400307DBE
:106200000F3E02287DD93236B07C401CB07416F89F
:106210003209E8B3306D03F087FB41EC100BFDF75A
:106220000BFED8F81000B0EE409AF0EE609A03F042
:1062300054F853EC192B03F0B7F841EC1A0B306DFE
:1062400003F072FB41EC100BFDF7AEFBD8F8140025
:10625000B0EE409AF0EE609A03F03FF853EC192B41
:1062600003F0A2F853EC1A2B03F074FA02F0D8FFF3
:10627000C8F84C00D8F84C00C01C03F02EF841ECD4
:10628000100BFDF7F5FB9FEDF71B53EC112B00E016
:1062900026E051EC100B02F02FFE02F0C1FF014688
:1062A000C8F85000D8F84C20D8F85400131A03222C
:1062B00093FBF2F21044C8F84C00C8F8540096F86A
:1062C0002D2090421EDD96F8440003281AD996F836
:1062D00046000844C1B24FF4FA70FEF77DFC84E634
:1062E00098ED050AD8ED040A96ED141AB8EEC00A26
:1062F000F8EEE00A00EEC10ABDEEC00A88ED130A0E
:10630000B8E705E0D948016821F0010101606CE6B9
:10631000D648016821F00101016066E696F82D106B
:10632000D8F848208A422BDDD8F86420B2EB410F20
:1063300026DD86F827B096F82810491CC9B286F8E1
:10634000281007290FD9C1B24FF4FA70FEF744FCA8
:1063500098ED0C0AF8EEC00A98ED0A0AB8EEC00AE9
:1063600002F0A4FB3073D8F84800B84204DD317B5A
:10637000B173C8F86C900746B07B3074307334E664
:10638000BA48016821F001010160D8F81000C8F88E
:106390002C00D8F81400C8F834000027C8F86CB0F6
:1063A00086F828B096F82700401C86F827001CE6DF
:1063B000D8F84000C8F82C00D8F84400C8F83400D9
:1063C0005F46C8F86CB016F8270F401C3070707B21
:1063D000273E012816D196F828000A2812D9D8F8A5
:1063E000781091FBF0F20A2A04DD4FF4FA60FEF710
:1063F0002DFC07E091FBF0F010F1140F02DAC82039
:10640000FEF724FCC8F878B086F834B086F828B0D7
:10641000EBE50121EEE50122F1E5FEF743FC96F8FC
:106420002700962801D1FEF771FC7079B24630B191
:106430009AF86C0000F01F0003287CD0DBE19AF88A
:106440006C008AF83F0000F00F018AF840103C28E9
:1064500003D1FCF7FFFECAF878009AF84000012843
:106460007FD19AF90C60D8F86C00C01C02F035FF9F
:1064700041EC100BFDF7FCFA9FED7D1B51EC100B6E
:1064800053EC112B03F066F902F0CAFE8146D8F8EE
:106490006C00C8F87000D8F84800412861DD8AF81F
:1064A0000D6096FBF9F000EBD07040108AF84500C3
:1064B0009AF90E009AF91010401AC01C02F00DFF54
:1064C00041EC100BFDF7D4FA51EC100B02F0A8FED2
:1064D0009AF9451091FBF0F040B28AF84500572E2A
:1064E00003DC9AF91010002904DA00EBD070401098
:1064F0008AF845009AF83B0000F133018E4209DB2F
:106500004030864206DC9AF9450000EBD07040101E
:106510008AF84500B9F1000F01DA8AF845B09AF916
:106520004500002801DA8AF845B09AF945000A28A2
:1065300005DD0A2001E05AE113E08AF845009AF9E6
:1065400045109AF90B000A1A032192FBF1F1084455
:106550008AF845008AF80B0016EB090F01D18AF87A
:1065600045B09AF8400002280CD19AF82B2042A19D
:106570004548DAF85830F9F735FF434A3A21032005
:10658000FEF770FC9AF81B0007280DD03E483FA18B
:10659000F9F728FF3C4A55210720FEF763FC3A4AE9
:1065A00014210720FEF75EFC9AF84000042828D149
:1065B000DAF878000A21B0FBF1F201FB1202B0FB1D
:1065C000F1F034A1CDE900029AF838309AF82C2085
:1065D0002D48F9F707FF2C4A3A210120FEF742FC2B
:1065E000D8F8740030A100909AF808209AF8293061
:1065F0002548521CF9F7F6FE234A3A210220FEF7FD
:1066000031FC9AF8400003280BD19AF8320068B1A7
:106610001D4828A1F9F7E6FE1B4A3A210420FEF79F
:1066200021FC9AF84000062805D054E0164823A122
:10663000F9F7D8FEF0E79AF8410004284BD09AF910
:106640000D20002A00DA52420F481EA1F9F7CAFEB7
:106650009AF90D00002839DB0B4A02210120FEF7D0
:106660008BFB38E0000000000000F83F0010004005
:10667000000000000000F03F4741494E25643C25E2
:10668000646D563E200000002802002444454D4F12
:106690000000000053253032642020462564252068
:1066A000206476256420000050256428256429256F
:1066B00064487A004742462E000000004742562EAA
:1066C000000000002530326400000000FE4A022174
:1066D0000120FEF78BFB9AF82600012804D09AF8D7
:1066E00040000B2848D049E09AF84100012804D026
:1066F000022820D0032821D057E09AF8400007282C
:1067000053D1D8F87000801000D54042C8F870000E
:10671000172802DD1720C8F8700098F870109AF951
:10672000110002F06BF840212046FEF767FFAA2017
:1067300002F09AF939E002F031FA36E098ED0C0AED
:10674000F8EEC00A98ED0A0AB8EEC00A02F0AEF9F7
:10675000C0EBC0010A2091FBF0F0B8F84810C1F37B
:10676000C70140B2FCF792F940210820FEF746FF2E
:10677000AA2002F079F918E0FEF7C8FAD8F860000C
:10678000002802DDC0B2FCF78DF8CF48CFA1F9F7A1
:1067900029FECD4A02210620FEF79AFB4021204621
:1067A000FEF72CFFAA2002F05FF99AF841000428B6
:1067B0000BD0062440212046FEF720FFAA2002F03D
:1067C00053F9641CE4B2082CF4D39AF840000F2863
:1067D0000CD1FBF754F853210420BDA2FEF742FB75
:1067E0009AF845008006000EFBF734F85EE3FBF7ED
:1067F00057F88AF818009AF8060020B101287DD0D1
:1068000002287CD052E3B34E9AF8010056F82020BB
:10681000AFF6CC01AC48F9F7E5FDAB4C0A21AA4A2A
:1068200017346078FEF754FB9AF83620AAA1A648E0
:10683000F9F7D8FD60785F21A34AFEF749FB9AF883
:106840000100801C56F82020AFF604119E48F9F78D
:10685000C9FDA0780A219C4AFEF73AFB9AF823204A
:106860009DA19948F9F7BEFDA0785F21964AFEF7F1
:106870002FFB9AF80100001D56F82020AFF63811C2
:106880009148F9F7AFFDE0780A218F4AFEF720FB27
:106890009AF94620012A04DA8B4891A1F9F7A2FD62
:1068A00003E0894890A1F9F79DFDE0785821864AD8
:1068B000FEF70EFB9AF80100801D56F82020AFF677
:1068C00078118148F9F78EFD20790A217E4AFEF77A
:1068D000FFFA9AF82E0087A1C0F106027A48F9F76C
:1068E00081FD20795F21784AFEF7F2FA9AF80100DB
:1068F000083056F82020AFF6B01101E051E160E217
:106900007148F9F76FFD60790A216F4AFEF7E0FAE6
:1069100070489AF839106838425C76A16A48F9F7ED
:1069200061FD60795F21684AFEF7D2FA9AF80100AA
:106930000A3056F82020AFF6F0116348F9F752FDFF
:10694000A0790A21604AFEF7C3FA9AF818306BA1C1
:106950009AF83A205C48F9F745FDA07931215A4A66
:10696000FEF7B6FA9AF801000C3056F82020AFF680
:1069700028215548F9F736FDE0790A21524AFEF7F9
:10698000A7FA9AF829205BA14F48F9F72BFDE07987
:1069900060214D4AFEF79CFA9AF801000E3056F835
:1069A0002020AFF65C214848F9F71CFD207A0A2127
:1069B000454AFEF78DFA9AF82A109AF8010000EB82
:1069C00041014448683050F82120AFF684213E4808
:1069D000F9F708FD207A32213B4AFEF779FA9AF856
:1069E0000100103056F82020AFF6A4213648F9F700
:1069F000F9FC607A0A21344AFEF76AFA9AF83020E4
:106A000041A13148F9F7EEFC607A5F212E4AFEF78A
:106A10005FFA9AF80100123056F82020AFF6D8211C
:106A20002948F9F7DFFCA07A0A21274AFEF750FA35
:106A30009AF8412028A12448F9F7D4FCA07A5F21D4
:106A4000214AFEF745FA9AF80100143056F8202042
:106A5000AFF60C311C48F9F7C5FCE07A0A211A4A56
:106A6000FEF736FA9AF81C201BA11748F9F7BAFC72
:106A7000E07A5F21144AFEF72BFA9AF801001630EB
:106A800056F82020AFF640310F48F9F7ABFC207BD9
:106A90000A210D4AFEF71CFA9AF82F0015A1C0F141
:106AA00009020948F9F79EFC207B5F21064AFEF7A0
:106AB0000FFA9AF8192016A10348F9F793FC607BA6
:106AC0000A21014A2CE000002802002450494E000F
:106AD000520000006C0100242D20256420000000DD
:106AE0002D282564292020002D282B2564292020ED
:106AF000000000002D2025642020000028256429A6
:106B0000202D2025642020002D2025642020200019
:106B1000464D20202020202D2025646D487A20001D
:106B2000FEF7D6F99AF81A00A8B3FF48FCA1F9F7C6
:106B300059FC607B1E21FC4AFEF7CAF99AF8010055
:106B4000183056F82020AFF60041F748F9F74AFC14
:106B5000A07B0A21F44AFEF7BBF90124012120465B
:106B6000F0A2FEF7B5F9A41CE4B2082CF6D39AF80B
:106B700025004FF0FF3101EB40018AF81E10042878
:106B800002D907208AF81E009AF81E000121E7A208
:106B9000FEF79EF98AE1FFE7E348E5A1F9F722FC59
:106BA000C7E79AF825000E388AF81E00DAF86C005C
:106BB00000F0070101297DD0DF4C9AF8010054F85C
:106BC0002020AFF67C41D848F9F70CFCD64A0A21C0
:106BD0000120FEF747F99AF80820D8A1D248521CA4
:106BE000F9F700FCD04A4B210120FEF73BF99AF857
:106BF0000100801C54F82020AFF6B441CA48F9F7D0
:106C0000F1FBC94A0A210220FEF72CF9DAF87800D4
:106C10000A21B0FBF1F201FB1203B0FBF1F2C24812
:106C2000C8A1F9F7DFFBC04A4B210220FEF71AF991
:106C30009AF80100001D54F82020AFF6F441BA483C
:106C4000F9F7D0FBB84A0A210320FEF70BF99AF8AE
:106C50002B20AFF27C11B448F9F7C4FBB24A4B21A8
:106C60000320FEF7FFF89AF80100801D54F8202059
:106C7000AFF62C51AC48F9F7B5FBAB4A0A2104201A
:106C8000FEF7F0F89AF81820B1A1A748D8F87430A8
:106C9000F9F7A8FBA44A2D210420FEF7E3F89AF89F
:106CA0000100083054F82020AFF664519E48F9F7EF
:106CB00099FB00E058E09C4A0A210520FEF7D2F833
:106CC0009948A7A1D8F85820F9F78CFB964A4B2190
:106CD0000520FEF7C7F89AF801000A3054F8202082
:106CE000AFF69C519048F9F77DFB8F4A0A210620A8
:106CF000FEF7B8F89AF801000C3054F82020AFF6EF
:106D0000B8518948F9F76EFB874A0A210720FEF738
:106D1000A9F89AF8320060B3834894A1F9F762FBAE
:106D2000814A4B210720FEF79DF89AF81B0007289F
:106D300024D07D488FA1F9F755FB7B4A0A21082012
:106D4000FEF790F801240121204676A2FEF78AF88A
:106D5000641CE4B2092CF6D39AF82500122812D04C
:106D6000002113281ED00FE0FAF79AFD8AF81800C8
:106D700022E76D4884A1F9F735FBD1E76A4884A181
:106D8000F9F730FBD9E701210022114316280BD077
:106D9000002001430AD09AF81E0001217FA2FEF7CD
:106DA00061F809E00122F0E70120F2E79AF81E00FD
:106DB00001215EA2FEF756F84FF6E850FDF7C2FF3C
:106DC00074E09AF83C0002287DD0FCF703FB052014
:106DD000FBF70AFE02460320FBF706FE42EA00200C
:106DE000CAF8700050486EA1F9F7FCFA01214E4A2A
:106DF0000846FEF76DF8DAF870306BA14A481A467B
:106E000003F50053F9F7EEFA474A59210120FEF73E
:106E10005FF89AF9122066A14348DAF87430F9F75E
:106E2000E1FA414A02210320FEF752F81E20FEF744
:106E3000FFFB9AF86C0000F00300022811D93A48D1
:106E400038A1F9F7CFFA9AF81D005A21364A0C38C2
:106E500001EBC000C1B20320FEF73AF83C20FEF778
:106E6000E7FB00242B212046FEF70DFA641CE4B258
:106E70007F2CF7D3534A54A12B48F9F7B3FA2A4A87
:106E800009210520FDF7EEFF274853A1F9F7AAFADB
:106E9000254A05210720FDF7E5FF234854A1F9F70E
:106EA000A1FA214A05210820FDF7DCFF5E46D14604
:106EB0008AF814B04FF40051DFF848A15046FAF7B1
:106EC000C6FE48B300E014E04FF480515046FAF794
:106ED000BEFE10B34FF480615046FAF7B8FE0028AA
:106EE0001CD04FF400615046FAF7B1FE002816D0CE
:106EF000CAE3FDF7EFFE0C4843A1F9F773FA0A4A1B
:106F000005210220FDF7E4FF2E4A074802F10C019B
:106F1000F9F768FA044A7FE0A9E063E1FDE3FDE3E5
:106F2000284F4E2920000000280200243E000000C7
:106F3000284F464629000000340100242D202564F6
:106F4000000000002D2025642E256420560000003E
:106F5000282564292D202564487A2020000000007F
:106F60002D20256420677220200000002D2047423C
:106F700046200000456E747279204B455920202030
:106F80002D2C2B20000000002D2047425620000011
:106F90004B4559204F4B2120202000006F0000005E
:106FA000436F6465202D3E002558255800000000E1
:106FB000456E742E4B65793C25643E20253034584F
:106FC00020000000A05A00083C53544D333248378B
:106FD0003E202573000000006D61696C3A207261EB
:106FE00064696F646F6D40692E7561202000000038
:106FF000687474703A20726164696F646F6D2E6F8B
:1070000072670000000402582020204B45592020C0
:107010004F4B2021200000001E210420FDF722FFFD
:10702000FE48FBA1DAF87020F9F7DCF9FB4A1D21D4
:107030000620FDF717FF9AF91300F9A100909AF9BD
:107040001230F648DAF87420F9F7CCF9F34A1D212A
:107050000720FDF707FF4FF4FA60FEF7E9FAFDF7A6
:1070600039FE8AF8065015208AF825001EE7DFF859
:10707000C483D8F8000020F00100C8F8000099F897
:107080002500FBF74BFB99F80300012845D140F69A
:10709000B830FDF7B9FD4FF4005850464146FAF7B5
:1070A000D6FD0028F9D0C82089F8280089F82700E3
:1070B00089F80360D8E31420FEF7BAFA99F81400AF
:1070C000401CC0B289F814000F2826D999F8050091
:1070D000C04389F80500FDF7FDFD89F8035089F8E4
:1070E0000A6099F8050090B199F8040089F8250024
:1070F000FAF7D6FB89F8180099F82500FBF70EFB84
:1071000089F806604FF47A70FDF77EFD0CE389F88C
:107110002560C820FEF78CFAF2E74FF40051504684
:10712000FAF795FD0028C6D099F80500F0B199F856
:10713000060001283ED0022848D099F82500401CBE
:10714000C0B289F825000E2801D989F8255099F890
:107150002500FBF7E3FA99F825000F2801D289F8FA
:1071600004004FF47A70FDF74FFDC1E689F81F5017
:10717000FDF7B0FDD8F8000020F00100C8F80000CD
:1071800099F82600401CC0B289F82600042801D1D5
:1071900089F82650FBF79EFB3220FEF749FA89F862
:1071A0001F50C820FEF744FAE62089F8280089F825
:1071B0002700D6E799F82500401CC0B289F82500C1
:1071C0001628C8D9162089F82500C4E799F82500A3
:1071D000401CC0B289F825001628BCD9162089F8B1
:1071E0002500B8E79349086820F00100086099F885
:1071F00025000C287DD009DC0C2887D2DFE800F0C0
:107200001F7979797979797979797979122871D0B1
:1072100008DCA0F10D010529EFD2DFE801F0F76AE3
:107220006A6A6A001528E5D004DC13287ED0142889
:107230007DD1FDE31628DDD04D28F9D1F9E3FDF726
:1072400049FD6420FAF7BEFD89F8355099F81B0016
:10725000072822D0714878A1F9F7C4F86F4A1E2197
:107260000220FDF735FE4FF44870FDF7CDFC4FF4DA
:107270006170FDF7C9FC4FF47A70FAF7A3FDFCE1E9
:107280002320FEF7D5F999F81400401CC0B289F804
:107290001400D9F86810884206D86A484FF4805123
:1072A000FAF7D5FC0028EBD099F81400D9F868104B
:1072B000884270D93220FAF785FD98ED050AF8EE7C
:1072C000C00A98ED040AB8EEC00A01F037FC89F84C
:1072D0000C00D8F81010D8F81400494300FB001037
:1072E00001F0FBFF41EC100BFCF70AFE51EC100B18
:1072F00001E0CAE185E201F093FF801001F0EDFFAB
:1073000041EC100BFCF7B4FB51EC100B01F0B8FF93
:10731000C4B20C2C00D90C2499F8320098B13F4823
:1073200049A1F9F75FF83D4A012101E081E2FBE163
:107330000846FDF7CDFD99F90C006FF0590A50454C
:1073400006DA012105E0354842A1F9F74BF8EAE7F2
:10735000002110F13C0F01DD012000E0002001437D
:1073600013D02E483EA1F9F73DF82C4A53210120B5
:10737000FDF7AEFD4FF49670FDF746FCC820FDF713
:1073800043FCBE20FDF740FC7EE0092C04D903201D
:1073900089F8380008E019E1062C03D9022089F8A1
:1073A000380001E089F838502FA11C48F9F71AF885
:1073B0001A4A53210120FDF78BFD4FF49670FDF71B
:1073C00023FC4FF4C870FAF7FDFC4FF41670FDF77C
:1073D0001BFC4FF4FA70FDF717FC99F90C0001F053
:1073E0007CFF53EC182B01F087FD41EC100BFCF7F0
:1073F000C7FD53EC102B9FED1D0B51EC100B01F052
:107400007BFD01F093FCC9F8500033E061E100001E
:10741000436F64653A202530345820002802002448
:107420004B65793A202025303458202825642D25B5
:1074300078290000001000402A2044454D4F202AA2
:107440000000000000040258477261756E6420421B
:10745000462D0000477261756E642042562D000073
:107460004572726F722100004F4B20000000000037
:107470000000F03F99F8320020B199F80C0089F82B
:10748000000001E089F800A0F8A1FE48F8F7AAFF83
:10749000FC4A02210620FDF7E5FC4FF44870FDF799
:1074A000B3FB8AE099F83800F7A10090224699F9D9
:1074B0000C30F448F8F796FFF24A01210420FDF75A
:1074C00007FDD9F8500002F02FFA41EC100BED48FF
:1074D000F2A153EC102BF8F785FFEA4A1E21082091
:1074E000FDF7C0FCF0484FF48061FAF7B0FB40BBF9
:1074F00099F80C00C846401C89F80C004FF4FA704B
:10750000FDF782FB98F90C0001F0E7FE53EC182B15
:1075100001F0F2FC41EC100BFCF732FD53EC102BA8
:107520001FED2E0B51EC100B01F0E6FC01F0FEFB01
:10753000C8F8500098F8320020B198F80C0088F88C
:10754000000001E088F800A04FF40061D648FAF787
:107550007EFB40BB99F80C00C846401E89F80C0021
:107560004FF41670FDF750FB98F90C0001F0B5FED2
:1075700053EC182B01F0C0FC41EC100BFCF700FDA4
:1075800053EC102B1FED470B51EC100B01F0B4FC2A
:1075900001F0CCFBC8F8500098F8320020B198F800
:1075A0000C0088F8000001E088F800A06420FAF7D9
:1075B00009FCBE494AF6AA2008604FF48051BA4837
:1075C000FAF745FB00283FF46DAF56E0D9F8588034
:1075D00089F8146089F8286089F8276089F81F50B5
:1075E00040F6E44AD04500DDD046A648B0A1424668
:1075F000F8F7F8FEA34A0A210320FDF769FC4FF4CF
:107600007A70FDF701FBB8F1C80F36DD9D48ADA1DA
:10761000F8F7E8FE9B4A05210720FDF723FC02202E
:10762000FEF706F8DFF880821FE04EF66020FDF7D7
:1076300089FB4FF400514046FAF709FBA8B94FF413
:10764000FA60FDF7E1FA42F21070FDF77BFBD9F822
:107650005820524500DD52468A4895A1F8F7C2FEEF
:10766000884A0A210320FDF733FC99F81400401CD6
:10767000C0B289F814001E28D7D389F83560C82015
:10768000FDF7D6FFFDF726FBF4E1401E10F0FF00EA
:1076900089F8250002D10E2089F8250099F82500E7
:1076A0000F2801D289F8040099F80610012904D1A5
:1076B0000E2802D1162089F825004FF44870FDF7F6
:1076C000A3FA99F82500FBF729F8C820FDF7B0FFC9
:1076D000D0E14FF4805842E01420FAF773FB99F898
:1076E0001400401CC0B289F81400D9F86810B0EB3F
:1076F000410F34D94FF47A70FDF786FA99F81A00E1
:10770000C8B189F81A604FF48040CAF81800042004
:10771000724988614FF4487001E064E2F9E3FDF7D3
:1077200073FA6420FDF784FF89F81F504FF49660C8
:10773000FDF76AFA9EE189F81A504FF08040CAF8C6
:1077400018000113654881613220FDF771FF99F837
:10775000190001F027F83220FDF76AFFDAE7414609
:107760005046FAF774FA0028B6D099F82500401E62
:1077700089F825001E20FDF75BFF7BE11920FDF74E
:1077800057FF99F81400401CC0B289F81400D9F8CA
:107790006810884235D94FF0000A89F8215001F06D
:1077A00031FA4FF095084FF41C7002901EE04C48DF
:1077B000C0F800800620FDF73BFFFAF771F850454E
:1077C00002DD8246C9F85480464890FBF8F0C117A4
:1077D00000EBD16044A142112A48F8F703FE294A80
:1077E00010210520FDF774FB08F10108029880457F
:1077F000DDDBFBF76FF84FF47A70FDF705FAFDF764
:1078000069FA29484FF48051FAF721FA0028B5D0D7
:1078100099F8210000288DD199F82500401E89F89B
:1078200025004FF49660FDF7EFF9C820FDF700FF43
:1078300020E1086820F00100086003E11920FDF74D
:10784000F7FE99F81400401CC0B289F81400D9F86A
:10785000681088427ED9FDF73DFA89F82150C8F8B2
:107860005860FBF7D7F845E01DE20000416D706CF1
:1078700069742E205068617365202046696C7472AB
:1078800000000000280200243C253032643E203CE9
:1078900025643E203C4625643E200000203C2530E7
:1078A0002E33663E20200000000402580048005895
:1078B0002A2A2A202564206D56202A2A2A202020C0
:1078C00020000000436F696C20626C2E707265733B
:1078D0007320274D656E75270000000000100258C8
:1078E0002C040040000E27072A20256420487A2017
:1078F0002A20200089F81F50F9A1FC48F8F772FDF2
:10790000FA4A0A210320FDF7E3FA4FF47A70FDF7F3
:107910007BF989F81F509621D9F868004843FDF794
:1079200087FEF248F2A1F8F75DFDF04A0A21032034
:10793000FDF7CEFA4FF44870FDF766F9D9F8680004
:1079400064214843FDF774FE4FF0000A002498EDCF
:10795000050A00E076E0F8EEC00A98ED040AB8EEF9
:10796000C00A01F0EBF88244C820FDF761FE641CF8
:10797000E4B20A2CEBD30A209AFBF0F05A304042D2
:10798000C8F85800B0F5B47F03DDA0F5B470C8F8AE
:107990005800D8F85800002803DA00F5B470C8F889
:1079A0005800FBF737F889F81F506421D9F86800B0
:1079B0004843FDF73DFE98ED050AF8EEC00A98ED44
:1079C000040AB8EEC00A01F0B9F8404301F085FCA2
:1079D00041EC100BFCF794FA9FEDC91B51EC100B16
:1079E00053EC112B01F0A4FC12D2C048C6A1F8F749
:1079F000F9FCBE4A0A210520FDF76AFAC820FDF706
:107A000003F99620FDF700F96420FDF7FDF813E077
:107A1000B648BFA1F8F7E6FCB44A0A210520FDF7F5
:107A200057FA4FF47A70FDF7EFF84FF4966001E0E3
:107A300021E02BE0FDF7E8F84FF44870FDF7F8FD82
:107A4000FDF748F9B4484FF48051FAF700F90028DF
:107A50003FF4F4AE99F8210000280BD199F82500E5
:107A6000401E89F825004FF47A70FDF7CDF8C82044
:107A7000FDF7DEFDFAE2401E89F825004FF496601E
:107A8000FDF7C2F8C820FDF7D3FDEFE24FF48058B0
:107A90000CE05020FDF7CCFD99F81400401CC0B25A
:107AA00089F81400D9F86810884205D84146504634
:107AB000FAF7CDF80028ECD099F81400D9F868103E
:107AC00088425AD9D9F87000FDF7CAFBD9F874106A
:107AD000884220D1F9F700FED9F8701088421AD1F7
:107AE00082488EA1F8F77EFC804A1E210320FDF714
:107AF000EFF94FF4FA70FDF787F84FF47A70FDF75D
:107B000083F88949B9F87400020A0A71887155200E
:107B100089F813001FE0754884A1F8F763FC734AE5
:107B200000210120FDF7D4F9704885A1F8F75AFC2F
:107B30006E4A00210320FDF7CBF96420FDF764F8BD
:107B40005020FDF761F86420FDF75EF899F8120007
:107B5000401C89F8120041465046FAF778F8002890
:107B6000F9D00120FBF7DCFB4FF4FA60FDF760FD74
:107B700078494FF48030886178E299F9120006283C
:107B80001DDA89F81460684899F81D10C23801445C
:107B900011F80C2D521C02F00F020A700278C17805
:107BA00041EA023142788078120242EA0010014331
:107BB000C9F874104FF49670FDF726F856E24B485A
:107BC00065A1F8F70FFC494A00210320FDF780F971
:107BD0006420FDF719F85020FDF716F84FF4FA600D
:107BE000FDF726FD42E2DFF884A1DAF8000020F07C
:107BF0000100CAF8000099F825000C286AD009DCB9
:107C00000C2866D2DFE800F01FB4C0CCD8E3FAF34A
:107C1000F2F1F0EF12285ED008DCA0F10D0005288B
:107C200057D2DFE800F0EAE9E8E7E600152853D08C
:107C300004DC132851D014284BD1BFE116284DD0B5
:107C40004D2846D1F6E1DFF8D0802DE01E20FAF76E
:107C5000B9F899F81400401CC0B289F81400D9F89A
:107C60006810B0EB410F1FD989F82150DAF80000F5
:107C700020F00100CAF8000099F82B00401CC0B2A7
:107C800089F82B00032801D189F82B504FF4487054
:107C9000FCF7BAFFC9F84C60C9F86C5089F81F505E
:107CA000C820FDF7C5FCD6E34FF480614046F9F7E4
:107CB000CEFF0028CAD099F8210050B999F82C00BD
:107CC000401CC0B289F82C001E2802D91E2089F859
:107CD0002C00BFE1E6E057E194E162E19DE10000A4
:107CE000204E6F2046657272697465002802002478
:107CF0002054616B652046657272697465000000EE
:107D00000000000000405540204572726F72210053
:107D1000204F4B210000000000040258204F4B214F
:107D2000202020202000000009010024207261642E
:107D3000696F646F6D40692E75612020200000001E
:107D400020202020204552524F5221202020202048
:107D5000200000000010025820204552524F5221AE
:107D6000204E3E3D35202120200000000010004024
:107D700099F83600401CC0B289F83600142802D9A0
:107D8000142089F8360065E199F82300401CC0B240
:107D900089F82300032802D9032089F8230059E138
:107DA00099F84600401C40B289F84600052802DDDB
:107DB000052089F846004DE199F82E00401EC0B21A
:107DC00089F82E00FF2801D189F82E6042E199F848
:107DD0003900401CC0B289F83900042802D90420B7
:107DE00089F8390036E151E044E02FE020E013E06B
:107DF00004E0BDE0A4E095E073E05EE099F83A00AD
:107E0000401CC0B289F83A00142802D9142089F81D
:107E10003A00FAF70BFE1DE199F82900401CC0B2A8
:107E200089F829000A2802D90A2089F8290011E1D5
:107E300099F82A00401CC0B289F82A00072802D904
:107E4000072089F82A00FBF79BF903E199F8300035
:107E5000401CC0B289F830000A2802D90A2089F8EB
:107E6000300099F8300040F2DC5110FB01F0F94984
:107E70004863EFE099F84100401CC0B289F8410026
:107E8000032802D9032089F84100E3E099F81C0097
:107E9000401CC0B289F81C005A2802D95A2089F81F
:107EA0001C00D7E099F82F00401EC0B289F82F00BF
:107EB000FF2801D189F82F60CCE099F81A00012839
:107EC0000ED199F81900401CC0B289F81900652834
:107ED00002D9652089F8190099F8190000F062FCB0
:107EE000B8E099F81B00072814D0FCF7F3FEAFF6B2
:107EF000B821D948F8F776FAD74A1E210320FCF7B3
:107F0000E7FFC820FCF780FE4FF4C870FDF790FB38
:107F1000A0E0ACE00120FBF7BDF94FF49670FCF750
:107F200073FE97E099F80800401CC0B289F8080079
:107F3000032802D9032089F80800FDF72DFB89E00A
:107F400099F83100401EC0B289F831001E2802D2D3
:107F50001E2089F83100FBF77DF9C9F8780047F257
:107F60003050FCF7EFFEFBF775F9C9F8780071E0C7
:107F700099F82B00401CC0B289F82B00022869D95F
:107F8000022089F82B0065E0D9F85400401EC9F89A
:107F90005400952802D29520C9F85400FAF79AFCAB
:107FA00058E0D8F85800401CC8F85800B0F5B47F25
:107FB00001DBC8F85860FAF72DFD4BE099F81B007B
:107FC000072814D0FCF786FEAFF69431A248F8F7E4
:107FD00009FAA14A1E210320FCF77AFFC820FCF70A
:107FE00013FEC820FDF724FBFCF774FE32E00120ED
:107FF000FBF750F99948FBF7B7F94FF49670FCF787
:1080000003FE27E099F83200401CC0B289F8320024
:1080100001281FD189F832501CE0022089F806009F
:108020004D2089F825004FF4FA70FCF7EDFDFCF7C0
:1080300051FE0FE099F81D00401CC0B289F81D00E8
:108040000F2802D90F2089F81D00FCF743FE3220CB
:10805000FDF7EEFA99F80A0018B94FF47A70FCF7B8
:10806000D3FD6420FDF7E4FA89F81F50F1E1DFF851
:10807000F0A1DAF8000020F00100CAF8000099F839
:1080800025000C286FD009DC0C2860D2DFE800F056
:108090001F606C7886929DAAB6C3D6EC12286ED06B
:1080A00008DCA0F10D00052851D2DFE800F0FAF855
:1080B000F7F6F50015286ED004DC13286CD01428D0
:1080C00045D16DE1162868D04D2840D1A5E14FF487
:1080D000006829E01E20F9F775FE99F81400401C8D
:1080E000C0B289F81400D9F86810B0EB410F1BD961
:1080F00089F82150DAF8000020F00100CAF80000E9
:1081000099F83800401CC0B289F83800032801D91A
:1081100089F83850C820FCF777FD0320C9F86C00B7
:10812000C820FDF785FA96E14E484146F9F78FFDE4
:108130000028CFD099F8210048B999F82C00401EAA
:1081400010F0FF0089F82C0001D189F82C5074E15F
:1081500099F83600401EC0B289F83600FF2801D1D8
:1081600089F8366069E18BE099F82300401E10F031
:10817000FF0089F8230001D189F823505DE1F4E084
:1081800099F84600401E40B289F84600002801DAFE
:1081900089F8466051E128E1F5E031E199F82E00D7
:1081A000401CC0B289F82E00062802D9062089F8A2
:1081B0002E0042E199F83900401E10F0FF0089F8C6
:1081C000390001D189F8395037E199F83A00401E59
:1081D000C0B289F83A00FF2801D189F83A60FAF76D
:1081E00025FC2AE199F82900401EC0B289F829002F
:1081F000032802D2032089F829001EE199F82A00F9
:10820000401EC0B289F82A00FF2801D189F82A60EF
:10821000FAF7B6FF11E199F83000401EC0B289F8B4
:108220003000FF2801D189F8306040F2DC5199F824
:10823000300010FB01F007494863FEE099F8410067
:10824000401E10F0FF0089F8410001D189F841502B
:10825000F3E009E0000800402802002408000024A0
:10826000001000400004025899F81C00401EC0B2E3
:1082700089F81C00502802D2502089F81C00DCE04C
:1082800099F82F00401CC0B289F82F00092802D9A4
:10829000092089F82F00D0E05CE043E035E014E0ED
:1082A000FFE799F81A0001280ED199F81900401E2D
:1082B000C0B289F81900582802D8592089F8190045
:1082C00099F8190000F06EFAB7E099F81B0007283A
:1082D00013D0FCF7FFFCAFF6A0618248F8F782F8F4
:1082E000804A1E210320FCF7F3FDC820FCF78CFC1C
:1082F0004FF4C870FDF79CF99FE00120FAF7CAFF20
:108300004FF49670FCF780FC97E099F80800401E47
:10831000C0B289F80800FF2801D189F80860FDF78C
:108320003BF98AE099F83100401CC0B289F831006D
:108330005A2802D95A2089F83100FAF78BFFC9F878
:10834000780047F23050FCF7FDFCFAF783FFC9F8DC
:10835000780072E099F82B00401E10F0FF0089F8B9
:108360002B006AD189F82B5067E0D9F854004FF4FC
:108370001C71401CC9F85400884201D9C9F8541036
:10838000FAF7A8FA59E0D8F85800401EC8F8580083
:1083900003D54FF4B470C8F85800FAF73BFB4CE033
:1083A00099F81B00072815D0FCF794FCAFF67871FC
:1083B0004C48F8F717F84B4A1E210320FCF788FDBC
:1083C000C820FCF721FC4FF4C870FDF731F9FCF729
:1083D00081FC32E00120FAF75DFF4348FAF7C4FF61
:1083E0004FF49670FCF710FC27E099F83200401E1D
:1083F000C0B289F83200FF281FD189F832601CE032
:10840000022089F806004D2089F825004FF4FA7003
:10841000FCF7FAFBFCF75EFC0FE099F81D00401E2C
:10842000C0B289F81D000C2802D20C2089F81D006A
:10843000FCF750FC6420FDF7FBF899F80A0018B926
:108440004FF44870FCF7E0FB6420FDF7F1F889F881
:108450001F5089F821600221DFF890804046F9F72B
:10846000F6FB30B34FF49670FDF7E2F80221404678
:10847000F9F7EDFBE8B1FCF72DFC1A481CA1F7F762
:10848000B1FF184A26210320FCF722FD4FF4167095
:10849000FCF7BAFB4FF4C870FCF7B6FBC820FCF73A
:1084A000B3FB4FF48030C8F8180041F28830FDF774
:1084B000BFF8D9F86C00401CC9F86C00B0F5E04F6B
:1084C0000AD3C9F86C60D9F85800B0F57A7F01D2A8
:1084D00089F81F50FCF71AFC07494AF6AA200860E1
:1084E000FDF768BC28020024080000240010025890
:1084F0003C204F4646203E000048005800B516205C
:10850000FAF766FA494A10740120FAF761FA907393
:10851000D0730220FAF75CFA02F8050C0320FAF790
:1085200057FA50740420FAF753FA90740520FAF7BA
:108530004FFAD0700620FAF74BFA50700720FAF77E
:1085400047FA90700820FAF743FA90710920FAF779
:108550003FFA10720A20FAF73BFA50760B20FAF72E
:1085600037FA02F80C0C1820FAF732FAD0710C2006
:10857000FAF72EFA90770D20FAF72AFA02F80F0C84
:108580000E20FAF725FA90750F20FAF721FA5072AB
:108590001220FAF71DFA03461120FAF719FA43EAF6
:1085A0000020D062283A5A2801D25A20506514205F
:1085B000FAF70EFA1D4B5833D8651320FAF708FA6C
:1085C00018B1D86D00F58070D8651520FAF700FA5B
:1085D00082F82C001F20FAF7FBF982F832001720EE
:1085E000FAF7F6F990760120FAF7FEF9D074022036
:1085F000FAF7FAF990740520FAF7F6F90346032022
:10860000FAF7F2F943EA002010670620FAF7ECF9CE
:1086100003460420FAF7E8F943EA002050670720F0
:10862000FAF7E2F982F8240000BD000028000024D7
:108630002DE9F0412DED028B4FF448735648014669
:1086400090F90C2091F822408031002A07DB0A279C
:108650008E6E92FBF7F5AD1D2E41F50717D0002A5F
:108660007EDA90F82F600D6EB54279DD6FF013055C
:1086700092FBF5F2C2F104058A6E2A41D2076FD14E
:1086800080F8432090F82A20022A48D057E0017F42
:108690008A427DDC90F8390001280FD0022815D0DD
:1086A000032831D0042873D1BDEC028B214602EBA4
:1086B000C200BDE8F0414000FCF78EBABDEC028B71
:1086C00021461846BDE8F041FCF786BA322A08DA9E
:1086D000BDEC028B21464FF4C870BDE8F041FCF7B9
:1086E0007BBA4A2A08DDBDEC028B214640F2DC5001
:1086F000BDE8F041FCF770BABDEC028B214618468C
:10870000BDE8F041FCF768BA92FBF7F0B421BDEC8C
:10871000028B48432146BDE8F041FCF75DBA90F872
:108720002B208C25896CA5EB42028A4207DDBDEC2B
:10873000028B21461846BDE8F041FCF74DBA90F88F
:108740002E00F6EE000A00EE100AB8EE400A20EE07
:10875000200A10EE100A01F0E7F89FED101B00E070
:1087600016E053EC112B00F013FB41EC180B2046E4
:1087700000F0CAFD53EC182B00F0BEFB00F080FDAA
:10878000BDEC028BC1B26420BDE8F041FCF724BA15
:10879000BDEC028BBDE8F081000000240000000069
:1087A0000000E03F10B54C3800F0AEFD9FED111B0E
:1087B00053EC112B00F0A0FB00F062FDC4B280214D
:1087C0000020FAF7E9FD4FF47A70FCF7BBFA31218B
:1087D0000020FAF7E1FDB9210220FAF7DDFD4B2177
:1087E0001020FAF7D9FD2146BDE810400120FAF724
:1087F000D3BD00009A9999999999A93F2DE9F04F15
:108800008846002844D000255A300A2190FBF1F018
:10881000C0EBC000401CC7B246464FF0800A4FF084
:10882000080917E0700700D100250AEB5500C5B212
:108830000124A9EBD60B3819C1B20BF0FF00FCF7ED
:10884000DDFE002000F010F9641CE4B2082CF2D325
:10885000761CF6B2182EE5D3002617E0700700D17B
:1088600000250AEB5500C5B20124A9EBD60B381937
:10887000C1B20BF0FF00FCF7C1FE284600F0F4F88F
:10888000641CE4B2082CF2D3761CF6B24645E5D35C
:10889000BDE8F08F0F490F4A91F82A1092F90C2089
:1088A000042901D1142A14DB002A01DA022910D08C
:1088B00002F146019D290CD20649002A91F82210A6
:1088C00003DD00F5FA70FCF787B9C0F5FA70FCF724
:1088D00083B97047000000242DE9F04105462DEDD5
:1088E000028B0024154E4FF4B4779FED138A04EBEE
:1088F000440000EBC4002844B84201DBA0F5B4708A
:1089000000EE100AB8EEC00A20EE080A10EE100AB7
:1089100001F00AF841EC100BFBF746F851EC100B94
:1089200000F004FA46F82400641C202CDFDBBDECC8
:10893000028BBDE8F08100002DFA8E3CD0020024AD
:108940002DE9F04105462DED028B0024154E4FF424
:10895000B4779FED138A04EB440000EBC400284475
:10896000B84201DBA0F5B47000EE100AB8EEC00A00
:1089700020EE080A10EE100A00F0D6FF41EC100BB2
:10898000FBF75AFA51EC100B00F0D0F946F824002E
:10899000641C202CDFDBBDEC028BBDE8F081000005
:1089A0002DFA8E3C500200242DE9F0412DED068B6E
:1089B00000241C4D9FED18AA9FED189B00F08DFC24
:1089C0000F46064600EE104A47EC186BB8EEC00A98
:1089D00020EE0A0A10EE100A00F0A6FF41EC100B80
:1089E000FBF72AFA53EC182B51EC100B00F0DCFCCF
:1089F00053EC182B00F0CCF953EC192B00F0C8F90C
:108A000000F03EFC45F82400641C202CDADBBDECB1
:108A1000068BBDE8F0810000F90F493E0000000020
:108A200000003E405004002410B50D4A4FF00041B4
:108A300091610C4B996100214FF4801494610306FD
:108A400002D50823936102E04FF4002393611023C1
:108A500093614006000E491CC9B20829EED310BD2F
:108A6000000402580000025810B54FF400410D4AAE
:108A70000B0493610C4B996100214FF480149461B5
:108A8000030602D50823936102E04FF400239361AB
:108A9000102393614006000E491CC9B20829EED389
:108AA00010BD0000000402580000025810B52DED62
:108AB000048BF0EE409AB0EE609A19EE100A00F0C6
:108AC00033FF1B4C41EC180BE07D00EE900AB8EE32
:108AD000601AC9EE010A30EEA90A10EE100A00F081
:108AE00023FF41EC100BB0EE481AF0EE681AFAF7CB
:108AF0005BFE9FED101B51EC100B53EC112B00F0A3
:108B000053FC00F08DFB94F82A10072900D10A309D
:108B100094F9001008445A305A2800DD5A206FF0AA
:108B20005901884200DA0846BDEC048B10BD0000F4
:108B3000000000246666666666A64C4010B52DED02
:108B4000048BB0EE409A10EE900A00F0EDFE41EC7E
:108B5000180B19EE100A00F0E7FE41EC100BB0EE16
:108B6000481AF0EE681AFAF71FFE9FED091B51EC48
:108B7000100B53EC112B00F017FC00F051FB0649D1
:108B800091F82A10072900D10A30BDEC048B10BDE2
:108B90006666666666A64C4000000024184BA3F18A
:108BA0008002986A92F82B10091D084140B2507556
:108BB0001B6B0B4159B2917501F116032C2B1DD87B
:108BC00000F13F037E2B19D892F90C30002B09DB02
:108BD000002900DA49420028C9B200DA404240B216
:108BE000F9F738BF002801DD40425075002900DA4E
:108BF000494292F91500C9B2F9F72CBF704700003D
:108C00008000002410B5FCF765F80B4806A1F7F7C3
:108C1000E9FB094A0A210320FCF75AF9BDE8104094
:108C20004FF4FA70FBF7F0BF20504C4541534520FC
:108C30005741495400000000280200241D4901F159
:108C4000EF008A7D82750A7D42704A754A7882708B
:108C5000CA7DC2700A7E02714A7A4271CA798271F3
:108C60000A7AC2710A7B02728A7B4272CA7F82725E
:108C700011F8062CC27291F82420027311F8092C05
:108C800042730A7F8273CA7BC2734A8E130A43748B
:108C90008274A0F191039A6DDA65130AC3740275A8
:108CA0008A7A427511F8082CC2754A7B0276097CD3
:108CB000C1777047220000240A4901F20910CA7CDA
:108CC00042708A7C8270B1F87020130AC3704271BE
:108CD000B1F87420130A0371827191F82410C171E4
:108CE000704700000000002410B500290AD0087861
:108CF000002807D005487844F8F7E0F8002801D0AC
:108D0000002010BD0248784410BD0000C6280000B5
:108D1000BE28000081F00041704780F0004070479D
:108D200021F00041704720F00040704721F00042E0
:108D3000A2F16052B2F5801F01F0004328BFD2F1CA
:108D40007F6C0BD95FEA001C43EAC20242EB507011
:108D500018BF704728BF20F001007047B2F5801F90
:108D6000BCBF184670474FEA410C1CF5001F02D2E9
:108D7000084600F04FBE70B500F0C0FB000000894F
:108D8000FFF7F6BF4FF00040A0F5800070470000ED
:108D900010B591EA030F48BF83F0004300F1E2846D
:108DA000841A71EB030C05D2121943EB0C03001B60
:108DB00061EB0C01DFF824E14FEA1154A4EB135CE2
:108DC0001EEA430F18BF9EEA445F73D023EA0E03E6
:108DD000DCF1200E21EA045143F4801332D322FA4D
:108DE0000CFE10EB0E0023FA0CFE41EB0E01CCF151
:108DF000200E03FA0EFE10EB0E0051F10001B1F54A
:108E0000801FCCF1200E32D201EB045112FA0EF287
:108E1000BDE8104058BF7047401C38BF5FEA4202AF
:108E200018BF7047002814BF20F0010041F1000175
:108E30004FEA410313F5001F38BF7047A1F1C0414D
:108E400000F0AABB012A43EB0302ACF1200CDCF1D9
:108E50001F0E32BF4FF0000E23FA0CF310EB03008D
:108E600041EB0451B4EB115FD0D0A1EB045101F5FB
:108E7000801149085FEA300001EB04510ED350F134
:108E8000000038BF12FA0EFE08D1BDE81040C9E755
:108E9000401C38BF5FEA4202CAD1C3E7BDE81040B8
:108EA0004FEA410313F5001F38BF7047A1F1C041DD
:108EB00000F072BB9EEA445F08D011EA5E0FBDE885
:108EC000104004BF01F0004100207047BDE8104091
:108ED00070B500F013FB00BF64FBBE3E0000E0FF76
:108EE000491058BFC1F140415B1058BFC3F1404326
:108EF0008B42EFF3008070472DE9C04130B4DFF8BA
:108F0000A0C23CEA111418BF3CEA131400F0EC8034
:108F100081EA03051CEA111444EAD57418BF1CEA5F
:108F2000131500F0C780A4EB05044FF0004545EA97
:108F3000C12145EAC32341EA505143EA525304F1A7
:108F40007F74994204F500344FEAC0204FEAC222F0
:108F500008BF904200F09C804FEA13650FF2401664
:108F6000765D4FEA134506FB05F7C7F1807706FBF0
:108F700007F74FEAD737A7FB03687642C8F5803872
:108F8000A7FB06CE38BFA8F1010807FB08E64FF0A3
:108F9000000EA6FB028CE6FB03CEDCF1000CCEF14A
:108FA000004E38BFAEF1010EA6FB0C584FF0000783
:108FB0004FF00005E6FB0E87A1FB08C6A0FB07CE1D
:108FC00016EB0E0645F10005E1FB076515F1E04ED5
:108FD0007EBFA4F580345FEA46066D4116F1800736
:108FE00045F100054FEA17274FEA066647EA05678D
:108FF000A6F1DE46B6F1805F4FEA15251FD9384647
:1090000024F0010C05EBC471BCF1FE6F01EB0C11F7
:1090100002D8F0BCBDE8008124425CBF01F5801E8F
:109020009EEAC47F02D4F0BCBDE80081244238D45B
:10903000F0BCA1F1C041BDE8004100F0ADBA4FEA7B
:10904000D22242EA43524FEAD323A7FB02864FEAD9
:10905000D02040EA415007FB03661EEA0E0F4FEA9C
:10906000D12105FB026658BFA6EB0056B6EB0056B1
:109070004FEA520E4EEAC37E18EB0E0E56EB530E1D
:10908000BDD518EB02085E417F1C55F10005B6E71F
:109090004FF480154FF000074FF000064FF0000826
:1090A000ADE7F0BC4FF0000001F1C04101F000411C
:1090B000BDE8008111EA0C1F0CEA131500D00CE08A
:1090C00013EA0C1F00F025804FF00000F0BC81EA8D
:1090D000030101F00041BDE80081F0BCBDE80041A2
:1090E00081EA030100F058BAF0BCBDE8004170B558
:1090F00000F004FA097EFC3E00F007B881EA0301A3
:109100004FF0000001F00041704781EA030100F0D8
:1091100043BAF0BCBDE800414FF000002149704760
:10912000FFFDFBF9F7F5F4F2F0EEEDEBE9E8E6E42C
:10913000E3E1E0DEDDDBDAD8D7D5D4D3D1D0CFCDB3
:10914000CCCBCAC8C7C6C5C4C2C1C0BFBEBDBCBBEC
:10915000BAB9B8B7B6B5B4B3B2B1B0AFAEADACABE7
:10916000AAA9A8A8A7A6A5A4A3A3A2A1A09F9F9EC1
:109170009D9C9C9B9A999998979796959594939373
:10918000929191908F8F8E8E8D8C8C8B8B8A89890A
:10919000888887878685858484838382828181808D
:1091A0000000FF070000F87F51EA030C17D41CF5FC
:1091B000801F58BFBCF5801F00F10680994218BF80
:1091C000704708BF9042704707D711F5801F58BFFE
:1091D00013F5801F19D499427047894270471CF5D6
:1091E000801F08D5BCF5801FF7D58B4218BF70478C
:1091F00008BF824270474FF4001C1CEB410F38BF80
:109200001CEB430F01D28B42704770B500F076F92A
:10921000922449004FF000514FF08053FFF760BE99
:109220004FEA41034FEA5353A3F58063D3F11E0382
:10923000C8BFD3F1210C0CDD4FF0004242EAC1223D
:1092400042EA505232FA03FC8CEAE17CACEBE1706A
:109250007047102BC4BF0020704703F5787CBCF129
:10926000FF3F04D06FF0004282EA2100704770B5E2
:1092700000F044F94992248000207047F2E7000092
:109280004FEA1153A3F58063D3F11E03A8BFD3F1B6
:10929000200C08DB4FF0004242EAC12252EA505251
:1092A00032FA03F0704709420BD4102BC4BF0020E0
:1092B000704703F5787CBCF1FF3F05D04FF0FF30DD
:1092C00070474FF00000704770B500F017F900BF0D
:1092D0004992248000207047F0E710F0004248BF18
:1092E0004042B0FA80F310FA03F10AD0C3F11D0333
:1092F00003F580634FEA415002EB035202EBD121A8
:1093000070474FF000007047B0FA80F310FA03F195
:109310000AD0C3F11D0303F580634FEA41504FEAC1
:10932000035202EBD12170474FF00000704700005C
:1093300051EA030C17D41CF5801F58BFBCF5801FE1
:1093400000F10680994218BF704708BF90427047ED
:1093500007D711F5801F58BF13F5801F19D4994204
:109360007047894270471CF5801F08D5BCF5801FE7
:10937000F7D58B4218BF704708BF824270474FF441
:10938000001C1CEB410F38BF1CEB430F01D28B427A
:10939000704770B500F0B2F8922449004FF00051C8
:1093A0004FF08053FFF79CBDDFF848C170B51CEA51
:1093B000111E1EBF1CEA13159EEA0C0F95EA0C0F36
:1093C00000F06F8081EA030423EA4C134EEAD47E56
:1093D00021EA4C1141F4801143F48013AE44A1FB07
:1093E000024CA0FB0365AEF17F7E361955EB0C05F0
:1093F000A1FB034C4CF10003A0FB021C16EB0C0676
:10940000654153F10003094218BF46F0010613F409
:10941000007F0BD14FEA03314FEA0530340341EAB4
:10942000155140EA16506FF003020AE04FEAC321DB
:109430004FEAC520F40241EA555140EA56506FF018
:10944000020202EB2E4201EB025585EACE710AD0F0
:109450005FEA440C18BF24F0004450F1000041F1D1
:10946000000120EAD47040F2FE7C624500D270BD5B
:10947000A84214BF4FF080444FF04044002E08BF74
:109480000024BEF1806FA8BFA1F1C041BDE87040CB
:1094900080F282804FF0000001F1C04101F00041F4
:1094A00070479EEA0C0F0CEA131518BF95EA0C0FD3
:1094B00006D04FF0000081EA030E0EF0004170BDAF
:1094C00000F01CF88900013E00F007B800F009B870
:1094D0004FEA430C5FEA5C5C08D081EA030100F0CC
:1094E0005BB84FEA410C5FEA5C5CF6D14FF00000DC
:1094F000014970470000FF070000F87F0EF1020EDF
:109500002EF0030E5EF8046B364205D4012A43EBBD
:10951000030515F5001F12D8012841EB010C1CF5BD
:10952000001F0CD80ED14FEAD17C15F5001F0CEBB3
:109530004C0C0CF1020C08BF4CEBD37C04E04FF058
:10954000080C01E04FEAD37C0CEB4C0526FA05F63B
:1095500006F00706B6F1040C06D20EEB860CBDE849
:1095600070404CF0010C6047DFE80CF0090B020280
:109570004FF000414FF00000A1F5002170BD1946E9
:109580001046012851EB010418BFD4F5001484BF24
:10959000002001F0004170BD0808A0F500114FEA5D
:1095A0003101704791EA030F10B581F000413FF59A
:1095B000F7AB83F0004300F0D5B800002DE9F0418F
:1095C00001F5801CBCF5001FC0F2A9804FEA115CB8
:1095D00021EA0C510CF1FD0C41F480115FEA5C0CA6
:1095E0000CF5C07C01D34000494130A4890241EA16
:1095F000905187028E0E0A0CA45D04FB04F602FB58
:1096000006F6C6F14046A4FB0662F60D46EA42267F
:1096100006FB06F4A4FB01235242C3F1404338BFCA
:109620005B1EA6FB02420024E6FB0324D20B42EAA7
:109630004446A6FB0623A1FB02E2A3FB07E4E3FBEF
:1096400061426442C2F1404E38BFAEF1010EA6FB4A
:1096500004234FF00002E6FB0E32A2FB0346340067
:10966000E2FB6264A1FB06E6A4FB07E8E4FB616899
:109670007642C8F1405838BFA8F10108A2FB06E4C1
:10968000A3FB08E5E2FB6854A1FB05E6A7FB04E8A1
:10969000E1FB648618F1200556F10006A809A8F13F
:1096A0001B08B10908F03F08B8F10A0F40EA8660CC
:1096B0001CD901EB0C51BDE8F08100BFFCF5EEE8D0
:1096C000E2DDD8D3CFCBC7C3C0BDB9B6B4B1AEAC61
:1096D000A9A7A5A3A19F9D9B9A9896959392908FD9
:1096E0008D8C8B898887868584838281A0FB006826
:1096F00000FB01F208EB4208B8EB872807D53418C5
:1097000058EB0104D5D5401C51F10001D1E7341AC2
:1097100078EB0104CDD4401E71F10001C9E75FEA86
:109720004C0C5FEA9C5C0DD105D34FF0000001F0BA
:109730000041BDE8F081BDE8F04170B5FFF7DEFE05
:109740006DDBFFBEBDE8F0414FF0000000497047FF
:109750000000F87F10B591EA030F48BF83F0004383
:109760003FF51EAB841A71EB030C07D212198CF073
:10977000004C43EB0C03001B61EB0C01DFF8A4E190
:109780004FEA1154A4EB135C1EEA430F18BF9EEA84
:10979000445F00F0B08023EA6E03524221EA045194
:1097A000C3EB6E0338BF5B1EDCF1200E25D322FA1B
:1097B0000CFE10EB0E0043FA0CFE41EB0E01CCF157
:1097C000200E03FA0EFE10EB0E0051F10001CCF159
:1097D000200E29D412FA0EF201EB0451BDE810401C
:1097E00058BF7047401C1CBFB2F1004F70470028A3
:1097F0000CBF491C20F00100704712EB020E43EB36
:10980000030218BF4FF0010E4EEA4202ACF1200CE9
:10981000DCF11E0E54D943FA0CFE10EB0E0051F190
:10982000FF31CCF11E0ED5D50EF1010E12FA0EFE4F
:10983000404141EB010101EB445C5FEA5C5C10D903
:1098400010EBDE7001EB045138BFBEF1004FBDE8F4
:10985000104018BF704700280CBF491C20F00100C1
:10986000704730D24FEAD42C11F5001124F4006473
:109870001BD0B1FA81F20B3AA41AA41ED2F1200334
:10988000914030FA03F31943904001EBCC71002C66
:1098900001EB0451BDE81040A8BF704701F1C04181
:1098A0004FF0000001F000417047B0FA80F310FA69
:1098B00003F100D110BDE41A173C4805C90AE4E7DA
:1098C00001EB045110BD491001EB0451BDE81040FB
:1098D0004FEA300002E04FF0000170474A0008BF35
:1098E0000042F8D0B2F5001F28BF704701F00041D8
:1098F0004FF0000070479EEA445F07D011EA5E0F08
:10990000BDE8104004BF002100207047BDE81040B2
:1099100070B5FFF7F3FD00BF40DFF63E83F0004176
:10992000104670470000E0FF43004FEAD30C4FEAB7
:109930003C0C43401FBF40070CF1605113F0FE4F39
:1099400070471CF0006F03D100200CF000417047FD
:109950000CF0004343EA507010B540EACC0000F030
:109960000EF800BF000000924FEA0001FFF714BE9E
:109970004FF000414FF00000A1F5002170470EF1BB
:10998000020E2EF0030E5EF8044B244204D44FEA7C
:109990004102B2F17F4F11D84FEA4003B3F17F4F3C
:1099A0000CD80ED14FEAD07CB2F17F4F0CEB4C0CAF
:1099B0000CF1020C08BF4CEBD17C04E04FF0080C1A
:1099C00001E04FEAD17C0CEB4C0324FA03F404F0E1
:1099D0000704B4F1040C06D20EEB840CBDE8104071
:1099E0004CF0010C6047DFE80CF0070802024FF072
:1099F0000040A0F5800010BD0846420018BFD2F11B
:109A0000807288BF00F0004010BD4FF04070E1EE62
:109A1000100A7047FF2141EAD050C0057047F6F7A1
:109A2000B0BF000000000404043C3C00000800003B
:109A30000008000800000000000000000000000016
:109A40000000000000000000000000000000000016
:109A50000000000000000000000000000000000006
:109A600000000000000000000000000000000000F6
:109A700000000000000000000000000000000000E6
:109A800000000000000000000000000000000000D6
:109A900000000000000000000000000000000000C6
:109AA0000000000000000000000000000000C0E016
:109AB000F0F8FCFCFCFCFCFCFCFCFCFCFCFCF8F006
:109AC000E0C000000000FFFFFFFFFFFF00000000FC
:109AD00000000000FFFFFFFFFFFF00000000FFFF8E
:109AE000FFFFFFFF0000000000000000FFFFFFFF7E
:109AF000FFFF00000000FFFFFFFFFFFF000000006E
:109B000000000000FFFFFFFFFFFF00000000030751
:109B10000F1F3F3F3F3F3F3F3F3F3F3F3F3F1F0FF5
:109B2000070300000000C0E0F0F8FCFCFCFCFCFCBB
:109B3000FCFCFC0000000000000000000000000031
:109B40000000000000FFFFFFFFFFFF00000000001B
:109B500000000000000000000000000000FFFFFF08
:109B6000FFFFFF00000000000000000000000000F8
:109B70000000000000FFFFFFFFFFFF0000000000EB
:109B8000000000000000000000000000003F3F3F18
:109B90003F3F3F0000000000000000000000C0E068
:109BA000F0F8FCFCFCFCFCFCFCFCFCFCFCFCF8F015
:109BB000E0C0000000000000000000000000000005
:109BC00000000000FFFFFFFFFFFF00000000C0E0FB
:109BD000F0F8FCFE7E7E7E7E7E7E7E7E7F3F1F0FC7
:109BE000070300000000FFFFFFFFFFFF0000000071
:109BF000000000000000000000000000000003075B
:109C00000F1F3F3F3F3F3F3F3F3F3F3F3F3F3E3CB8
:109C10003830000000000C1C3C7CFCFCFCFCFCFC14
:109C2000FCFCFCFCFCFCF8F0E0C0000000000000C4
:109C3000000000000000000000000000FFFFFFFF28
:109C4000FFFF00000000000000007E7E7E7E7E7E22
:109C50007E7E7E7EFFFFFFFFE7C300000000000066
:109C6000000000000000000000000000FFFFFFFFF8
:109C7000FFFF0000000030383C3E3F3F3F3F3F3F8A
:109C80003F3F3F3F3F3F1F0F070300000000FCFC2A
:109C9000F8F0E0C00000000000000000C0E0F0F8B4
:109CA000FCFC00000000FFFFFFFFFFFF00000000C2
:109CB00000000000FFFFFFFFFFFF00000000070F94
:109CC0001F3F7F7F7E7E7E7E7E7E7E7EFFFFFFFF4C
:109CD000FFFF000000000000000000000000000086
:109CE00000000000FFFFFFFFFFFF0000000000007A
:109CF00000000000000000000000000003070F1F2C
:109D00003F3F00000000C0E0F0F8FCFCFCFCFCFC65
:109D1000FCFCFCFCFCFC7C3C1C0C00000000FFFF7D
:109D2000FFFFFFFF00000000000000000000000037
:109D3000000000000000070F1F3F7F7F7E7E7E7EB9
:109D40007E7E7E7EFEFEFCF8F0E00000000000005B
:109D5000000000000000000000000000FFFFFFFF07
:109D6000FFFF0000000003070F1F3F3F3F3F3F3F43
:109D70003F3F3F3F3F3F1F0F070300000000C0E091
:109D8000F0F8FCFCFCFCFCFCFCFCFCFCFCFC7C3C63
:109D90001C0C00000000FFFFFFFFFFFF00000000A1
:109DA0000000000000000000000000000000FFFFB5
:109DB000FFFFFFFF7E7E7E7E7E7E7E7EFEFEFCF8C7
:109DC000F0E000000000FFFFFFFFFFFF00000000C9
:109DD00000000000FFFFFFFFFFFF0000000003077F
:109DE0000F1F3F3F3F3F3F3F3F3F3F3F3F3F1F0F23
:109DF0000703000000000C1C3C7CFCFCFCFCFCFC91
:109E0000FCFCFCFCFCFCF8F0E0C0000000000000E2
:109E1000000000000000000000000000FFFFFFFF46
:109E2000FFFF000000000000000000000000000034
:109E300000000000FFFFFFFFFFFF00000000000028
:109E4000000000000000000000000000FFFFFFFF16
:109E5000FFFF000000000000000000000000000004
:109E60000000000003070F1F3F3F00000000C0E09C
:109E7000F0F8FCFCFCFCFCFCFCFCFCFCFCFCF8F042
:109E8000E0C000000000FFFFFFFFFFFF0000000038
:109E900000000000FFFFFFFFFFFF00000000C3E71E
:109EA000FFFFFFFF7E7E7E7E7E7E7E7EFFFFFFFFCA
:109EB000E7C300000000FFFFFFFFFFFF00000000FE
:109EC00000000000FFFFFFFFFFFF0000000003078E
:109ED0000F1F3F3F3F3F3F3F3F3F3F3F3F3F1F0F32
:109EE000070300000000C0E0F0F8FCFCFCFCFCFCF8
:109EF000FCFCFCFCFCFCF8F0E0C000000000FFFFF4
:109F0000FFFFFFFF0000000000000000FFFFFFFF59
:109F1000FFFF00000000070F1F3F7F7F7E7E7E7ED9
:109F20007E7E7E7EFFFFFFFFFFFF0000000000003F
:109F3000000000000000000000000000FFFFFFFF25
:109F4000FFFF0000000030383C3E3F3F3F3F3F3FB7
:109F50003F3F3F3F3F3F1F0F07030000000000004F
:109F600000000000000000000000000000000000F1
:109F700000000000000000000000000000000000E1
:109F800000000000000000000000000000000000D1
:109F900000000000000000000000000000000000C1
:109FA00000000000000000000000000000000000B1
:109FB00000000000000000000000000000000000A1
:109FC0000000000000000000000000000000000091
:109FD0000000000000000000000000000000000081
:109FE0000000000000000000000000000000000071
:109FF0000000000000000000000000000000000061
:10A000000000000000000000000000000000000050
:10A010000000000000000000000000000000000040
:10A020000000000000000000000000000000000030
:10A030000000000000000000000000000000000020
:10A040000000000000000000000000000000000010
:10A050000000000000000000000000000000000000
:10A0600000000000000000000000000000000000F0
:10A0700000000000000000000000000000000000E0
:10A0800000000000000000000000000000000000D0
:10A0900000000000000000000000000000000000C0
:10A0A00000000000000000000000000000000000B0
:10A0B00000000000000000000000000000000000A0
:10A0C0000000000000000000000000000000000090
:10A0D00000000000000038FCFC3800000000000D0B
:10A0E0000D000000000E1E00001E0E00000000000B
:10A0F0000000000020F8F820F8F82000020F0F02FE
:10A100000F0F0200387C444747CC9800060C0838F3
:10A11000380F070030300080C06030000C060301AB
:10A12000000C0C0080D87CE4BCD84000070F080865
:10A13000070F080000101E0E0000000000000000C5
:10A14000000000000000F0F80C040000000003070D
:10A150000C0800000000040CF8F000000000080CDF
:10A160000703000080A0E0C0C0E0A080000203015F
:10A1700001030200008080E0E08080000000000316
:10A180000300000000000000000000000000101E9E
:10A190000E00000080808080808080000000000031
:10A1A0000000000000000000000000000000000CA3
:10A1B0000C00000000000080C06030000C060301AD
:10A1C00000000000F8F80CC40CF8F00003070C08BD
:10A1D0000C070300001018FCFC0000000008080F2A
:10A1E0000F080800080C84C4643C18000E0F09080E
:10A1F000080C0C00080C444444FCB800040C08088B
:10A20000080F0700C0E0B098FCFC800000000008C8
:10A210000F0F08007C7C444444C48400040C0808EC
:10A22000080F0700F0F84C4444C08000070F0808EE
:10A23000080F07000C0C0484C47C3C0000000F0FC6
:10A2400000000000B8FC444444FCB800070F0808B4
:10A25000080F0700387C444444FCF8000008080854
:10A260000C07030000000030300000000000000672
:10A270000600000000000030300000000000080E62
:10A28000060000000080C0603018080000000103D4
:10A29000060C0800002020202020200000010101E1
:10A2A000010101000008183060C0800000080C06A1
:10A2B00003010000181C04C4E43C18000000000D59
:10A2C0000D000000F0F008C8C8F8F000070F080BF8
:10A2D0000B0B0100E0F0988C98F0E0000F0F0000ED
:10A2E000000F0F0004FCFC4444FCB800080F0F08EA
:10A2F000080F0700F0F80C04040C180003070C0802
:10A30000080C060004FCFC040CF8F000080F0F0811
:10A310000C07030004FCFC44E40C1C00080F0F08AD
:10A32000080C0E0004FCFC44E40C1C00080F0F0891
:10A3300000000000F0F80C84848C980003070C08DF
:10A3400008070F00FCFC404040FCFC000F0F000021
:10A35000000F0F00000004FCFC0400000000080FC8
:10A360000F08000000000004FCFC0400070F0808B0
:10A370000F07000004FCFCC0E03C1C00080F0F00AD
:10A38000010F0E0004FCFC0400000000080F0F0881
:10A39000080C0E00FCFC387038FCFC000F0F0000AD
:10A3A000000F0F00FCFC3870E0FCFC000F0F0000F9
:10A3B000000F0F00F8FC040404FCF800070F080865
:10A3C000080F070004FCFC44447C3800080F0F0809
:10A3D00000000000F8FC040404FCF800070F080E5D
:10A3E0003C3F270004FCFC44C4FC3800080F0F006D
:10A3F000000F0F00183C6444C49C1800060E0808A7
:10A40000080F0700001C0CFCFC0C1C000000080FCF
:10A410000F080000FCFC000000FCFC00070F08080F
:10A42000080F0700FCFC000000FCFC000103060C08
:10A4300006030100FCFC000000FCFC00070F0E03FB
:10A440000E0F07000C3CF0E0F03C0C000C0F030179
:10A45000030F0C00000C7CC0C07C3C000000080F07
:10A460000F0800001C0C84C4643C1C000E0F09087B
:10A47000080C0E000000FCFC0404000000000F0F9C
:10A48000080800003870E0C08000000000000001F3
:10A4900003070E0000000404FCFC00000000080894
:10A4A0000F0F0000080C0603060C08000000000057
:10A4B000000000000000000000000000202020201C
:10A4C00020202020000003070400000000000000FE
:10A4D0000000000000A0A0A0E0C00000070F0808D6
:10A4E000070F080004FCFC2060C08000000F0F086C
:10A4F000080F0700C0E0202020604000070F080878
:10A50000080C040080C06024FCFC0000070F080851
:10A51000070F0800C0E0A0A0A0E0C000070F0808D7
:10A52000080C040040F8FC440C180000080F0F0849
:10A5300000000000C0E02020C0E02000276F484855
:10A540007F3F000004FCFC4020E0C000080F0F002B
:10A55000000F0F00000020ECEC0000000000080FCE
:10A560000F0800000000000020ECEC0000307040FC
:10A57000407F3F0004FCFC80C0602000080F0F01FA
:10A58000030E0C00000004FCFC0000000000080F9B
:10A590000F080000E0E060C060E0C0000F0F00079F
:10A5A000000F0F0020E0C02020E0C000000F0F00CF
:10A5B000000F0F00C0E0202020E0C000070F0808B7
:10A5C000080F070020E0C02020E0C000407F7F4847
:10A5D000080F0700C0E02020C0E02000070F084857
:10A5E0007F7F400020E0C06020E0C000080F0F081F
:10A5F0000000000040E0A02020604000040C090999
:10A600000B0E04002020F8FC202000000000070FA3
:10A61000080C0400E0E00000E0E00000070F08087C
:10A62000070F080000E0E00000E0E0000003070C76
:10A630000C070300E0E0008000E0E000070F0C07DB
:10A640000C0F07002060C080C0602000080C0703CA
:10A65000070C0800E0E0000000E0E000474F484839
:10A66000683F1F00606020A0E06020000C0E0B0916
:10A67000080C0C00004040F8BC0404000000000777
:10A680000F080800000000BCBC0000000000000F24
:10A690000F000000000404BCF84040000008080F50
:10A6A00007000000080C040C080C04000000000067
:10A6B00000000000E0F0988C98F0E0000F0F000020
:10A6C000000F0F0004FCFC4444CC8C00080F0F0862
:10A6D000080F070004FCFC4444FCB800080F0F08F6
:10A6E000080F070004FCFC04040C0C00080F0F0802
:10A6F0000000000000F8FC0CFCF800001C0F0F0824
:10A700000F0F1C0004FCFC44E40C1C00080F0F0895
:10A71000080C0E000C3CE0FCE03C0C000C0F010FA0
:10A72000010F0C00080C444444FCB800040C080859
:10A73000080F0700FCFC80C060FCFC000F0F01004C
:10A74000000F0F00FCFC80C260FCFC000F0F01003A
:10A75000000F0F0004FCFCC0E03C1C00080F0F00C1
:10A76000010F0E0000F0F81C0CFCFC00080F0F009D
:10A77000000F0F00FCFC387038FCFC000F0F0000CD
:10A78000000F0F00FCFC404040FCFC000F0F0000DD
:10A79000000F0F00F8FC040404FCF800070F080881
:10A7A000080F0700FCFC040404FCFC000F0F000071
:10A7B000000F0F0004FCFC44447C3800080F0F0815
:10A7C00000000000F0F80C04040C180003070C084B
:10A7D000080C0600001C0CFCFC0C1C000000080F00
:10A7E0000F0800001C3C60C080FCFC0000000C0D49
:10A7F00007030100F0F808FC08F8F0000103020F5D
:10A80000020301000C3CF0E0F03C0C000C0F0301D3
:10A81000030F0C00FCFC0000FCFC00000F0F0808FC
:10A820000F1F1800387CC08080FCFC000000000076
:10A83000000F0F00FC00FCFC00FC00000F080F0FD5
:10A84000080F0000FC00FCFC00FC00000F080F0FCC
:10A85000081F180004FCFC4040C0C000080F0F088F
:10A86000080C0F00FCFC40C0C000FC000F0F080CDF
:10A870000F000F0000FCFC4040C0C000000F0F089C
:10A88000080C0F000C0404C4CCF8F0000C080808F5
:10A890000C070300FCFC80F80404F8000F0F00070D
:10A8A000080807000078CC8484FCFC00080C060330
:10A8B000010F0F0000A0A0A0E0C00000070F0808D3
:10A8C000070F0800E0E02020202000000F0F0909FA
:10A8D00009060000E0E0A0A0A04000000F0F08085B
:10A8E00008070000E0E02020206000000F0F0000BB
:10A8F0000000000000E02020E00000001C0F0C0C15
:10A900000F1C0000C0E0A0A0A0E0C000070F0808D6
:10A91000080C040020E080E080E02000080F010F18
:10A92000010F0800402020A0E06000000408090991
:10A9300006060000E0E0000080E000000F0F0201CA
:10A94000000F0000E0E0001080E000000F0F0201A7
:10A95000000F000004FCFC80C0602000080F0F0105
:10A96000030E0C0000E02020E0E0000008070000DB
:10A970000F0F0000E0C00000C0E000000F00010168
:10A98000000F0000E0E00000E0E000000F0F010118
:10A990000F0F0000C0E0202020E0C000070F0808D3
:10A9A000080F0700E0E02020E0E000000F0F0000AB
:10A9B0000F0F000020E0C02020E0C000407F7F4853
:10A9C000080F0700C0E0202020604000070F0808A3
:10A9D000080C04002020E0E02020000000000F0F01
:10A9E0000000000060C08000E0E000000C0C0703E5
:10A9F00001000000C020F0F020C0000003040F0F91
:10AA0000040300002060C080C0602000080C070321
:10AA1000070C0800E0E0000000E000000F0F08084D
:10AA2000080F1800E0E00000E0E00000010302026F
:10AA30000F0F0000E000E0E000E000000F080F0F43
:10AA4000080F0000E000E0E000E000000F080F0F3A
:10AA5000081F1000000000000000000000000000BF
:10AA600000000000E080800000E000000F08080700
:10AA7000000F000080808080808080000000000047
:10AA80000000000040202020E0C000000408080969
:10AA90000F070000E000C02020C000000F010708E1
:10AAA00008070000C0202020E0E0000008050301A6
:10AAB0000F0F000000000000000000000000000078
:10AAC00000000000000000000000002F0000000750
:10AAD000000700147F147F14242A7F2A12231308EE
:10AAE000646236495522500005030000001C2241D3
:10AAF000000041221C0014083E081408083E080803
:10AB00000000A0600008080808080060600000203D
:10AB1000100804023E5149453E00427F4000426118
:10AB20005149462141454B311814127F10274545A4
:10AB300045393C4A494930017109050336494949BB
:10AB400036064949291E00363600000056360000F8
:10AB50000814224100141414141400412214080291
:10AB600001510906324959513E7C1211127C7F492C
:10AB70004949363E414141227F4141221C7F49499A
:10AB800049417F090909013E4149497A7F0808087E
:10AB90007F00417F41002040413F017F0814224156
:10ABA0007F404040407F020C027F7F0408107F3EC0
:10ABB0004141413E7F090909063E4151215E7F091D
:10ABC000192946464949493101017F01013F404069
:10ABD000403F1F2040201F3F4038403F631408146F
:10ABE0006307087008076151494543007F414100F0
:10ABF00001060830400041417F0004020102044088
:10AC000040404040000305000020545454787F48E1
:10AC10004444383844444420384444487F385454E9
:10AC20005418087E09010218A4A4A47C7F08040417
:10AC30007800447D40004080847D007F10284400DF
:10AC400000417F40007C041804787C0804047838B4
:10AC500044444438FC2424241818242418FC7C0878
:10AC60000404084854545420043F4440203C4040CD
:10AC7000207C1C2040201C3C4030403C44281028B4
:10AC8000441CA0A0A07C4464544C4400107C82006E
:10AC90000000FF000000827C100008040810087CFF
:10ACA0001211127C7F494949317F4545453A7F0160
:10ACB000010103603F213F607F49494941730C7F97
:10ACC0000C732141494D337F1008047F7E20110809
:10ACD0007E7F08142241403F01017F7F0608067FE6
:10ACE0007F0808087F3E4141413E7F0101017F7F8F
:10ACF000090909063E4141412203017F0103612602
:10AD00001806011C227F221C63140814633F2020B4
:10AD10003F60070808087F7F407F407F3F203F203B
:10AD20007F017F4848307F4878007F7F4848300067
:10AD30004149492A1C7F103E413E661909097F207E
:10AD4000545478403E494545387E4A4A34007C0494
:10AD5000040C00384545493E38545454184C307C56
:10AD6000304C24424A34007C20107C007C21117C31
:10AD7000007C10284400403C04047C7C0810087CC3
:10AD80007C10107C0038444444387C04047C00FC73
:10AD900018242418384444442804047C04044C90A7
:10ADA00090907C18247E241844281028443C2020AD
:10ADB0003C601C10107C007C407C407C3C203C2093
:10ADC0007C047C5070007C5070007C7C50700000D3
:10ADD000424252523C7C10384438402C127E0000D3
:10ADE0000000000048DB3DB412C05CB5A00F19B6EE
:10ADF00005AD8FB6CDF866B604B1543771E29C3814
:10AE0000C336743923C4023A679A193A435766BA6B
:10AE1000896506BCE5E102BD71A1BDBD86EC5EBEE3
:10AE2000F533333F86EC5EBE71A1BDBDE5E102BDE9
:10AE3000896506BC435766BA679A193A23C4023A31
:10AE4000C336743971E29C3804B15437CDF866B614
:10AE500005AD8FB6A00F19B612C05CB548DB3DB486
:10AE600067A029BD9C5775BD6FD1A5BD4AC9D4BD8A
:10AE7000F8C102BEE1D3533FF8C102BE4AC9D4BDF6
:10AE80006FD1A5BD9C5775BD67A029BD84B46FBDAA
:10AE90005893B5BDDB14FCBD17B123BE66BE5D3F44
:10AEA00017B123BEDB14FCBD5893B5BD84B46FBD90
:10AEB00014BEA1BD6FEDFCBDDC252FBEE9383F3FC0
:10AEC000DC252FBE6FEDFCBD14BEA1BD5BC0FF3CF9
:10AED00045D0BF3D45D0BF3D5BC0FF3C0000803F3B
:10AEE000D417A5BFF8782A3FE66401BE10D2AC3E65
:10AEF00010D2AC3E00000000000000000000803FC7
:10AF0000E05BA6BE000000000000000030313233DC
:10AF1000343536373839414243444546403058008D
:10AF200030313233343536373839616263646566BF
:10AF3000403078000400000800000000000000021B
:10AF4000000100001000000004FA97999999D93F78
:10AF5000AF788E1DC571CC3F9FC678D0099AC33F8C
:10AF6000935555555555E53F599322942449D23F61
:10AF7000DE03CB966446C73F44523EDF12F1C23F28
:10AF80004FBB610567ACDD3F182D4454FB21E93F01
:10AF90009BF681D20B73EF3F182D4454FB21F93FF0
:10AFA000E2652F227F2B7A3C075C143326A6813C76
:10AFB000BDCBF07A8807703C075C143326A6913C21
:10AFC000C4EB98999999C9BF711623FEC671BCBF8D
:10AFD0006D9A74AFF2B0B3BF9AFDDE522DDEADBFF5
:10AFE0002F6C6A2C44B4A2BF0D5555555555D53F0D
:10AFF000FF8300922449C23F6E204CC5CD45B73F28
:10B00000513DD0A0660DB13FEB0D76244B7BA93F9F
:10B0100011DA22E33AAD903F4C5555555555A53FB1
:10B020007751C1166CC156BF9015CB19A001FA3EDD
:10B03000AD529C804F7E92BEC4B1B4BD9EEE213E07
:10B04000D43888BEE9FAA8BD000000000000000066
:10B0500000004054FB21F93F3163621A61B4D03DD6
:10B060000000601A61B4D03D7370032E8A19A33BAF
:10B070000000002E8A19A33BC14920259A837B3901
:10B0800000000000000000006E83F9A22915444E64
:10B09000D15727FCC0DD34F5999562DB4190433CE4
:10B0A000AB6351FE61C5BBDE3A6E24B7E0D24D42C0
:10B0B000EA2E49061C92D1091CEB1DFE3EA729B1C0
:10B0C000F53582E88444BB2E26709CE9417E5FB44E
:10B0D00039D69139F43953838B5F849C3B28F9BD71
:10B0E000FF97F81F0F9805DE8B112FEF1F6D0A5A7F
:10B0F000CF7E366DB709CB27663F464F2DEA5F9E60
:10B10000C7BA27757BF1E5EBF739073DEA92528A1A
:10B11000B15FFB6B085D8D1FA6F810111111813F07
:10B12000D561C119A0012ABF7DFEB157E31DC73EFD
:10B13000EB9C2B8AE6E55ABE7CD5CF5A3AD9E53D41
:10B140007AFE10111111C13F37D60684F464963F80
:10B15000280356C9226D6D3F0165F2F2D844433F82
:10B16000A69237A0887E143F735360DBCB75F3BE85
:10B17000FE41B31BBAA1AB3F93846EE9E326823F45
:10B180001583E0FEC8DB573F68108D1AF726303F65
:10B19000E9A7F0320FB8123FD47ABF74702AFB3E91
:10B1A00002400000000000A0000000000540000078
:10B1B000000000C8000000000C4000000000409C9F
:10B1C00000000000194000000020BCBE000000008C
:10B1D00034400000BFC91B8E00000004B5400000D1
:10B1E000504BCFD06607E2CF010000006C41000059
:10B1F0003E8251AADFEEA73401000000D9420000D0
:10B20000DCB5A0E23A301F97FFFFFFFFB445000016
:10B21000FD25A0C8E9A3C14FFFFFFFFFFF3F0000CE
:10B220000000008000000000FF3F000000000080E0
:10B2300000000000564F4C2E4645202020202000C4
:10B2400053454E532046452020202000564F4C5554
:10B250004D45202020200000444953504C455920A2
:10B260002020200020204649454C4420202000007A
:10B2700020205041524B202020000000564F4C2EE1
:10B28000544F4E4520200000484F542053544F4EF9
:10B290004520200020204245414348202000000056
:10B2A00046494C544552204C50202000504F5745A1
:10B2B000522020004C454420425249474854202007
:10B2C0000000000057524954452020202D206F7265
:10B2D000202B2000444953432D200000564F4C2E74
:10B2E000572E5349472E2000414C4C204D45544188
:10B2F0004C322000564F4C2E534348454D452000BC
:10B30000205255424249534820000000414C4C20F5
:10B310004D4554414C2000002043752B41672B20A4
:10B320002A0000005752495445202D206F72202BCF
:10B3300000000000465245512E000000D093D180FD
:10B340002ED0A1D0BB2ED0A1D0B8D0B32E000000FB
:10B350003000000050524F46494C4500464552527D
:10B36000495445004742562F474246005059432F03
:10B37000454E470020536561424541434800000067
:10B380004741494E00000000424154544552590083
:10B39000D09CD095D094D0ACD18AD0BFD0BBD18E28
:10B3A000D1810000D0ADD09AD0A0D090D09DD18ACC
:10B3B000D18AD18AD18AD18A00000000D0A4D09845
:10B3C000D09BD0ACD0A2D0A0D18AD18AD18AD18A48
:10B3D000D18A0000D18AD18AD18AD09FD09ED09BB9
:10B3E000D095D18AD18AD18AD18A0000D0AFD0A09D
:10B3F000D09AD09ED0A1D0A2D0ACD18AD18AD18A05
:10B40000D18A0000D0A2D09ED09DD18AD097D09270
:10B41000D0A3D09AD090D18AD18AD18A00000000DE
:10B42000D18AD18AD18AD09FD09BD0AFD096D18AF1
:10B43000D18AD18A00000000D0A2D09ED09AD18AB1
:10B44000D18AD18A00000000D18AD18AD18AD09FC6
:10B45000D090D0A0D09AD18AD18AD18A00000000A1
:10B46000D093D09ED0A0D18AD09AD090D09CD09D9D
:10B47000D098D18AD18A0000D0A7D0A3D092D0A1F1
:10B48000D0A2D18AD096D095D09BD18AD18A000003
:10B49000D18AD18AD18AD09CD0A3D0A1D09ED0A06D
:10B4A000D18AD18A00000000D093D0A0D09ED09C39
:10B4B000D09AD09ED0A1D0A2D0ACD18AD18A00009F
:10B4C000D09CD09ED0A0D0A1D09AD18AD09FD09B22
:10B4D000D0AFD096D18A0000D090D0A2D090D09A90
:10B4E000D090D18AD093D0A0D09ED09CD18A000099
:10B4F000D091D090D09BD090D09DD0A1D18A000087
:10B50000D094D098D0A1D09AD18C0000D0A7D0A34D
:10B51000D09220D096D095D09BD095D097D0900047
:10B52000D091D095D097D18AD096D095D09BD095F8
:10B53000D097D09000000000D0A7D090D0A1D0A28A
:10B54000D09ED0A2D0900000D0A4D095D0A0D0A002
:10B55000D098D0A200000000D0A7D090D0A1D0A257
:10B5600000000000D092D0A1D095D18AD09CD09577
:10B57000D0A2D090D09BD0AB00000000D09FD0A034
:10B58000D09ED0A4D098D09BD0AC0000D091D090C9
:10B59000D0A2D090D0A0D095D0AF0000D8B50008F0
:10B5A0000000002428020000D4020008C0B60008F1
:10B5B00028020024780F0000300300081C0000005F
:10B5C00043000000F8FFFFFF0C0000000E00000029
:10B5D0000F0000002E00000032A662015907013E54
:10B5E00005B00AD7A3BC7F0102040A5A13C2160190
:10B5F0000208010815010501571764015001011FD8
:10B6000014B414019303B41354B314087CB51B0889
:10B6100088081A8C081A80081A38081A34081A5828
:10B62000081A5C081A48081A240813F0B41B0864A6
:10B63000081A6C04134CB21B08A8101AF4081AD884
:10B64000081ADC081A3C181A34081A78101A7C08F0
:10B650001A04081AAC081A38081AA0081ABC201ACA
:10B66000D4081119501AB4082AEC6419081AA4084D
:10B670001A88081A60281A40081A0C201AC4081AD6
:10B6800050181A0C041A64101AE8101A20081A64C8
:10B69000081AD4142A941019301A740C1AC00811FC
:10B6A00019081A90081A70181A48082A181019044C
:10B6B000113C90D00304400880C0E0F0F8FCFE008C
:040000050800029954
:00000001FF
